:020000020000FC
:02000000EEC050
:02000800567828
:100034000C946C2E0C946A2E4156522D43686970B0
:100044004261736963322028632920323030362DAF
:1000540032303039204A6F65726720576F6C667290
:04006400616D0000CA
:10007000C4EDD1E00895C0E1D1E00895C0E0D1E041
:100080000895CCE3DDE00895E0E0F6EF0895E0E0C8
:10009000F6EF0895FF91EF91EF93FF93EF2FE85460
:1000A000F2E4FA5FE650E8F7EE2708950093340192
:1000B0000895009134010895009346010895009138
:1000C000460108950093170108950C9405360C9489
:1000D000A1310C9410320C9431310C948C310C946D
:1000E000BB330C949A330C94A2330C94CC340C9400
:1000F000213C0C94DF310C942E360C943536409113
:100100001C01089540911E01089540911F0108951A
:1001100040911D0108950C94BF370C94CB370C947B
:10012000DB370C94B6360C94D03C0C94AD3C0C945C
:10013000CE330C94D0350C94F4340C9416350C94C6
:10014000373A0C947E3A0C94E3380C94C8380C94EB
:10015000D4380C94F2370C9445380C94C13A0C9472
:10016000EA3A0C94B43A0C94DD3A0C940E360C94A2
:10017000233D0C94363D0C94F13C0C94ED3C0C94D6
:10018000F73C0C94FC3C0C94F33C0C94413D0C94D7
:10019000633D0C946C3D0C94823D0C94893D0C9411
:1001A000DB3E0C94BF3F0C9432400C94A8400C945E
:1001B0004E400C94623F0C94A93D0C94B73D0C94B6
:1001C000413F0E942A400C94003E0E94CC3D0C947A
:1001D000BC3E0E94863E0C94E83D0C942E3EF89462
:1001E000A0E02A2EA1E03A2EA0E1AEBFAFEFADBF56
:1001F0000E9424300E94E63C0E940E790E945838EA
:100200000E94A131AFEFA0930801A0933901209281
:100210004501209246012092580188277894209227
:100220003501A0913101A4FD0C942F010E94A13150
:100230000E9404040E942E36D2CFAF91BF91CF917D
:10024000DF91EF91FF9108950F901F90FF93EF932F
:10025000DF93CF93FF93EF931F920F920895A1E046
:100260000E940E31AA270E949E309927A7E10E9482
:1002700009310E94A131A0E10E940931C4E0DAE015
:10028000E7E3F7E10E941635A7E00E9409310E94DA
:10029000A2330704200030D1A6E10E940931C5E055
:1002A000D8E0E6E0F9E00E941635D8E1F9E10E94D5
:1002B0001635D8E0F9E0CC5FEC5FC833A0F368E70F
:1002C0000E94053640911C0141FD0EC06A95C1F7A0
:1002D00056E142E00E94213C0E9405360E9405360C
:1002E0005A95B9F70C9491010E94A1310E94A23352
:1002F00000004B6579626F6172642D546573740000
:100300000E94DF3170917D01A0917D01A215E1F382
:1003100020927D0190E07A2F0E948C310E940F3252
:10032000F3CFA0E00E940E31A1E00E94AB379927E5
:1003300020923201AA270E949E30A5E10E94093135
:100340000E94A131C0E0D0E0EDE1F4E10E946A3505
:10035000A1E50E9409310E94A233010183838383B6
:100360008383204156522D436869704261736963EB
:1003700032208282828282820000A5EAB4E00AE40E
:100380000D9304EC0D930CE80D9308E20D9302E637
:100390000D9306EA0D93509606EA0D9302E60D932F
:1003A00008E20D930CE80D9304EC0D930AE40D9311
:1003B0009DD2409145014B3008F0442740934501C0
:1003C000642F67FD66276B3008F06AE050E06F939A
:1003D000A6D06F9153955830D1F761D136D10BD15A
:1003E0006F9387D16F91423E11F46A95EACF433EF5
:1003F00011F46395E6CF443E21F4643010F064506C
:10040000E0CF453E21F4673010F46C5FDACF6830FE
:10041000F8F04A3E11F0443F19F760934501683007
:1004200039F44A3EE9F676D00E94DD1D73D079CFCB
:10043000693039F44A3EA1F66DD00E94AA226AD0F2
:1004400070CF68D04A3E61F60E944A2463D069CFDB
:100450004F9340911C0142FD2AC04F914A3E11F03A
:10046000443F41F46093450155D088270E9404041D
:1004700051D057CF413F41F4609345014BD088277D
:100480000E94EA0347D04DCF423F39F460934501C3
:1004900041D00E948B1F3ED044CF433F39F460933C
:1004A000450138D00E94F21F35D03BCF99CF4F91F4
:1004B000413F39F4609345012DD00E948F032AD02B
:1004C00030CF423F39F46093450124D00E94EE249E
:1004D00021D027CF433F39F4609345011BD00E94C0
:1004E000292518D01ECF443F09F76093450112D04B
:1004F0000E94D7030FD015CF0E94A233FF4156525E
:100500002D436869704261736963322056302E3919
:1005100033000895A0911E01A030E1F70895A1E0F5
:10052000B3E050FDA95F51FDA25F52FDBA5F452FB8
:100530000E94B979042F4EE20E3409F44CE265179B
:1005400009F44295409334010E94BB330E94A233C8
:10055000FF20200040E50E941032452F4F5C0E9492
:1005600010320E94A233FF202000B3950E94BB33BB
:10057000452F0E94B9794E3481F40E94A233FF20A6
:1005800020E6E7202000B3950E94BB330E94A233EF
:10059000FF2020E8E92020000FC00E94A233FF20A6
:1005A00020D0D1202000B3950E94BB330E94A233FB
:1005B000FF2020D2D3202000452F0E942B7AB39514
:1005C0000E94BB3366E045910E9410326A95D9F7CC
:1005D000B3950E94BB3366E045910E9410326A9544
:1005E000D9F7B3950E94BB330E94A233FF2020208D
:1005F0002020200008954AE26A3009F44295409391
:1006000034010E94A2330F0F202020202020000060
:100610000E94A233100F2020D4D5202000000E9479
:10062000A233110F2020D6D7202000000E94A23331
:10063000120F20494E464F2000000E94A233130F94
:100640002020202020200000089548E2693009F48D
:100650004295409334010E94A2330F0820202020AD
:10066000202000000E94A23310082020D8D920208A
:1006700000000E94A23311082020DADB20200000B5
:100680000E94A2331208434F4E46494700000E9481
:10069000A2331308202020202020000008954CE2DF
:1006A000683009F44295409334010E94A2330F014F
:1006B00020202020202000000E94A23310012020B2
:1006C000DCDD202000000E94A23311012020DEDFAB
:1006D000202000000E94A233120144464C4153489E
:1006E00000000E94A23313012020202020200000BF
:1006F00008953DED20921F010E94F13640911C01AA
:100700004470431739F0342F403011F4EFD0F4CF58
:1007100008D1F2CF40911F01403071F30895A4E059
:100720000E940931C1E0DFE0ECE1F3E10E946A35AB
:10073000A0E40E9409310E94A2331002436F707935
:100740002050726F6772616D20746F007091450167
:1007500060E0ACE0671709F4A0E60E940931B2E15D
:10076000A62FAA0FA60FAD5F0E94BB3340E50E94E3
:100770001032462F47704F5C0E94103263956830EC
:1007800041F70E942E36423E21F47030D1F37A9523
:10079000DFCF433E21F47730A1F37395D9CF4A3EA2
:1007A00019F40E945E7A08954D3E59F708950E940B
:1007B000DD3A4F436C656172207468697320507232
:1007C0006F6772616D3F2000413009F008950E940B
:1007D000387A0895A0911E01A030E1F70E94B77900
:1007E0004E3441F00E94150520923501A0911F0161
:1007F000A43F09F096CD08D00E943536A0E00E94B3
:100800009E300E94A131E6CF0E94A131882720921C
:100810001E010E94297A3C9645914E3429F4339664
:10082000F695E79509957DCD0E94D50E209215018C
:1008300020925801209232010E94DF31A7E20E94EB
:10084000093192E0A0914601A03079F0A33021F463
:10085000A7E20E94093109C0A0E10E940931A0E489
:10086000A0930001A0EEA0930101A0914601A03049
:1008700051F40E94A2331600205052455353204594
:10088000534320002EC0A13051F40E94A2336900CE
:1008900020505245535320455343200022C0A230DC
:1008A00051F40E94A2334200205052455353204538
:1008B0005343200016C0A33049F40E94A2332F00F6
:1008C000205052455353204553432000A53069F42E
:1008D0000E94A233380020505245535320455343C1
:1008E0002000A0911E01AD3EE1F70895A0E00E9416
:1008F00009310E94A2331500202020202020202032
:1009000020202020202020202020202020202020E7
:100910002020202020200000ECE2F9E00E94453851
:100920000895EAE4F9E00E94453808952020202047
:100930002020204564697420205361766520204C76
:100940006F6164202052756E2020202020202020FE
:1009500020436F7079202053656E642020526563B8
:10096000762020436C656172AA270E940E31A3E0B5
:100970000E94AB378F93409145010E9424790E94D9
:10098000A1310E949330992740911E014030E1F738
:100990000E94A23300002050524F4752414D200088
:1009A000409145014F5C0E9410324AE30E94103290
:1009B000CFEDD1E058D2F0D20E94F879EBD38F91ED
:1009C000A8E8803069F1ACECEEECF1E1813031F077
:1009D000ABE48A9545914030E9F7F8CF4CD292E0EC
:1009E000A5E0B1E00E94BB330E949A330E94A2337B
:1009F000FF20494E20500000409142014F5C0E9470
:100A000010324AE30E941032BB27AC2DA3950E94FE
:100A100031314AE30E941032AD2DA3950E9431314D
:100A20000895AAE25A2E70E208959927FADF9CDF12
:100A3000D22CAA27BB27D09236010E9458360E949A
:100A4000F136403E11F4AA27F6CF413E11F4AFE152
:100A50002BC0423E11F4AA9527C0433E69F4A395EA
:100A60009B2F0E94220A9A1730F4BE3511F4AA95E2
:100A70001BC0AA27B39518C0443E21F4BA95B7FD10
:100A8000BB2712C0463E21F4B850B7FDBB270CC0AF
:100A9000473E11F4B85F08C0453E11F4B39504C059
:100AA0004A3E39F5B395AA27A03838F0AFE1BA9598
:100AB000B038C0F0AA27BB27BECFA03228F0BE3581
:100AC00089F0AA27B395B7CFBF3508F0BEE50B2F45
:100AD0000D1508F4D02E0D2D015F0B1718F40B2FF8
:100AE0000F50D02E9B2F0E94220A9A1708F4A92F8C
:100AF000A2CF9B2F4E3E39F4AF93BF930E94E409DF
:100B0000BF91AF9189C14F3E31F4BF930E94EF096D
:100B1000BF91AA2781C1493E11F482D17DC14C3ECB
:100B200031F4A03009F489CFAA957AD175C15091DA
:100B30001C01547009F4C5C0433FD1F4ACEC9BD107
:100B40000E94A23301075245434549564520505261
:100B50004F4752414D20592F4E203F006DD12EF46A
:100B600075D218D35EDF5092D4017DD1882761CF32
:100B7000423F39F5ACEC7FD10E94A23301075345C7
:100B80004E442050524F4752414D20592F4E203F46
:100B9000000052D156F7ACEC6ED10E94A23301078F
:100BA00053454E44494E472E2E2E202020202020F3
:100BB000202000003092320193D12092320131DFA7
:100BC000D4CF443FB1F4ACEC56D10E94A23301071C
:100BD000434C4541522050524F4752414D20592FCE
:100BE0004E203F0029D126F4C3D21BDF5092D401FE
:100BF000BCCF413F41F5ACEC3ED10E94A23301078E
:100C00005052494E542050524F4752414D20592F77
:100C10004E203F0011D1B6F4ABE42DD10E94A23397
:100C200001075052494E54494E472E2E2E20202067
:100C3000202020202000A2E0A093320151D1209258
:100C40003201EFDE92CF433671F462E46093F1013A
:100C500065E56093F20166E46093F3016DE36093F0
:100C6000F40161D2EACE483791F462E46093F10175
:100C700065E56093F20166E46093F3016DE36093D0
:100C8000F4010E94930864D25092D40118C04637F0
:100C9000B1F46091F101623499F460E26093F10182
:100CA0006093F2016093F3016093F4016093F501A6
:100CB0006093F6012BD26ED25092D401BECE88271B
:100CC000BCCE423F11F5BF93AF93C9D0D9F0ACEC85
:100CD000D2D00E94A2330107534156452050524FB3
:100CE0004752414D20592F4E203F0000A5D046F4D9
:100CF0000E94C4790E94F8794DD293DE7093D4019A
:100D0000B2D08827AF91BF9196CE433FE1F4BF9315
:100D1000AF93A5D0B9F0ACECAED00E94A2330107DE
:100D20004C4F5354204348414E47455320592F4E72
:100D3000203F000081D026F70E94F8792BD271DE87
:100D40007093D401DDCF413F49F46A2E7B2EADD0A4
:100D5000A62DB72D5092D40170CED2CF4D3E09F5BD
:100D6000BF93AF937CD0A9F0ACEC85D00E94A233A6
:100D700001075155495420572F4F205341564520C4
:100D8000592F4E203F0058D046F7A0911E01A030A9
:100D9000E1F70E948B30A0E00E949E30AF91BF919E
:100DA0000895443FE1F45BD029F40E948B300E9407
:100DB000A1310895A9E65FD00E94A23301075341F3
:100DC0005645204348414E474553204245464F52E1
:100DD000452052554E2100000E942E3691CF509151
:100DE0001C0152FD1CC053FD1AC04C31C0F04038EC
:100DF000B0F4AF3171F05A2FAFE10E94AD366A9175
:100E00006983AA95A517D9F74883A3955092D40171
:100E100014CE0E94AD3648835092D4010ECE0DCE32
:100E20000E94AD365A2F5F3121F049814993539585
:100E3000FACF50E2588308950E942E36493559F072
:100E4000493749F04A3E39F04E3439F04E3629F0F0
:100E50004D3E19F0F1CF68940895E8940895A0915B
:100E6000D401A0320895A8E806D00E94A23301055B
:100E70004F4B00000895EF93FF939927A0934801EB
:100E80000E94A233010520202020202020202020A5
:100E90002020202020202020202020202020202052
:100EA00020202000FF91EF910895A0E00E9480365D
:100EB0004A3E09F40895423E21F4A030B9F3AA95C0
:100EC000F5CF433E21F4AB3089F3A395EFCF403209
:100ED00068F3403858F74883AB3009F0A395E6CF64
:100EE000C5EDD1E056E149910E9410325A95D9F7EB
:100EF0000E94DF314EE511D016F04A95E1F7542FEC
:100F000053954427451719F024D04395FBCF43E26E
:100F10000E9410320E94DF310895CF93DF935F93D8
:100F20006F93E894C0E4D2E053E2459FC00DD11D19
:100F300050E26991613238F45A95D9F76F915F9117
:100F4000DF91CF91089568946F915F91DF91CF9178
:100F50000895DF93CF934F935F936F93CDE3D2E0E8
:100F600053E2459FC00DD11DDF93CF93A39653E26B
:100F70006A91613210F45A95D9F7CF91DF91499176
:100F80000E9410325A95D9F70E94DF316F915F911C
:100F90004F91CF91DF910895AF93BF93EF93FF935C
:100FA0004F93E0ECFFE0AAE1B2E04591403011F050
:100FB0004D93FBCF4F91FF91EF91BF91AF9108956A
:100FC00020457869742020204E616D6520202053D3
:100FD000617665202052656C6F6164202020527517
:100FE0006E202000AF93BF93EF93FF934F93E4EFF6
:100FF000FFE0D9CF20202020202020205072696ED1
:1010000074202053656E6420202052656376202072
:1010100020204E6577202000AF93BF93EF93FF937E
:101020004F93E8E2F0E1BFCF2041626F727420205D
:1010300020202020202020202020202020202020B0
:10104000202020202020202020202000E5DFACECE4
:1010500012DF0E94A2330105524543454956494ECD
:10106000472E2E2E0000209236010E94B8089927A4
:10107000ECECE0934801EFEDF1E0EE2EFF2E41E1C4
:101080000E94BF375CE00E94DB374B31B9F14A3335
:10109000D1F70E94DB374B3189F1403218F0419390
:1010A0005A95B9F7403228F00E94DB374B3131F1C5
:1010B000F9CFEAE1F2E0EE2EFF2E53E2EE2DFF2D06
:1010C000B396EE2EFF2E0E94DB374B31B9F0403243
:1010D000D0F3433299F006C00E94DB374B3171F0F8
:1010E000403248F041935A95B9F70E94DB374B31B3
:1010F00029F04032D0F793959036F9F60895A3E29F
:10110000BA9FADE3B2E0A00DB11D0895BF93AF93B8
:10111000F6DFC4E8D1E053E249914D935A95E1F7E7
:10112000AF91BF910895BF93AF93E9DFC4E8D1E0D9
:1011300053E24D9149935A95E1F7409184014093D0
:10114000F501409185014093F601AF91BF9108955B
:10115000BF93AF934F935F93D2DF139640E250E279
:101160004D935A95E9F75F914F91AF91BF910895D3
:10117000DF93CF93BF93AF934F9340E2ADE3B2E0E1
:10118000CDEFDCE04D932197E9F74F91AF91BF91FF
:10119000CF91DF91DF93CF93BF93AF934F9341E014
:1011A000ADE3B2E0C0E3D42FDA5010F0C395FCCF2A
:1011B000D65CCD93DD93C0E2CD93909643954036B7
:1011C00089F74F91AF91BF91CF91DF91089542522E
:1011D00045414B004F564552464C4F5700444956E7
:1011E000494445202F30005351522046524F4D2044
:1011F0003C3000434F4E5354414E5420544F4F20E7
:101200004249470057524F4E472045585052455388
:1012100053494F4E0053594E544158204552524F56
:101220005200554E4B4E4F574E204B4559574F523B
:10123000440057524F4E4720464F524D41540042B2
:101240004144204C494E454E554D424552004E4575
:10125000585420572F4F20464F5200524554555254
:101260004E20572F4F20474F53554200544F4F2089
:101270004D414E5920474F53554200544F4F204D3A
:10128000414E5920464F5200493243204552524F59
:101290005200554E4B4E4F574E204552524F520022
:1012A00044464C415348204552524F52004F5554EA
:1012B000204F4620415252415900494E434F4D5014
:1012C0004C45544520504152004B4559574F5244CC
:1012D000204953204D495353494E470057524F4ED2
:1012E000472042434F505920004F5554204F46202D
:1012F00053435245454E0043414E4E4F54204352B6
:10130000454154452046494C45004D454D4F5259A5
:101310002046554C4C0046494C45204E4F542046E3
:101320004F554E440050414745204E4F5420494EA2
:101330002046494C45005041474553204E4F5420CC
:10134000494E2052414E4745004E4F5420494E20B1
:101350004752415048494353204D4F4445004E4F5A
:101360005420494E2054455854204D4F4445004E7A
:101370004F205553522046494C4500535243204F6D
:101380005554204F462053435245454E0044455343
:1013900054204F5554204F462053435245454E004C
:1013A00057524F4E47205350524954450057524FC1
:1013B0004E4720454550524F4D20414452004E4F1C
:1013C000204558544D454D00BE3508F00895BF9353
:1013D00028D0B395BE35E1F7BBDEBF91DBCEBE357D
:1013E00008F00895BF93AF93AB2FAA95BDE508D041
:1013F000BA95BA17E1F7B395ABDEAF91BF91CACEFC
:10140000BF93AF93DF93CF937ADE1396ED01B0E2F3
:10141000A991AAA3BA95E1F7CF91DF91AF91BF91BE
:101420000895BF93AF93DF93CF9369DE1396ED01D9
:10143000B0E2ABA1A993BA95E1F7CF91DF91AF915B
:10144000BF910895BF93AF93DF93CF9358DEED0123
:1014500093964E914132E8F34038D8F7AC1BBC0B61
:101460009A2F925097FD9927CF91DF91AF91BF911D
:101470000895C6EFDCE02A922A9280E02F92AA27F4
:10148000BB27442771917032E9F37C3121F4A1919B
:10149000BB27719156C07E3121F4A191BB27719178
:1014A00050C07D3121F4B191A19171914AC07F3139
:1014B00021F4B191A191719144C07C3130F4572F46
:1014C0004C2E5D2ECE2FDF2F63C07432C1F471918C
:1014D000703320F07A3310F4705305C0713468F023
:1014E000773458F47753B03148F4A295B2955A2F17
:1014F0005F70A07FB52BA70FEACF23C029C0703340
:1015000050F17A3340F5403810F086E030C1AA0F30
:10151000BB1FF0F04A2E5B2EAA0FBB1FC8F0AA0F0C
:10152000BB1FB0F0A40DB51D98F07053A70FB21DEE
:1015300078F0B7FD0DC07191703318F07A3308F46C
:10154000E6CF4F3709F479D1AA93BA9340E89DCFFB
:1015500085E00DC144C07134E8F37B35D8F7608174
:10156000613458F16B3548F54C2E5D2ECE2FDF2FB0
:1015700021970C2F1D2FE4E4FDE152E075917030AE
:1015800011F488E0F4C0703261F46991683299F422
:101590005F93452FAA27BB27EC2FFD2FC42DD52DF8
:1015A00071CF6991671751F375917032E9F75395CF
:1015B000C02FD12FE3CF87E0DAC0403810F086E0AB
:1015C000D6C07154770FEF93FF93ECE9FCE0E70F7F
:1015D000F21DA191B191FF91EF917191B2CF7D3246
:1015E00051F44F3711F444274DCF20F4403210F01E
:1015F0004FE748CF75C0783231F471E07F93AA2766
:10160000BB27472F3FCF793209F064C05F9151303B
:1016100019F0523011F409D159C0533011F419D1D5
:1016200055C0543029F4D2D1803009F0A0C04CC04C
:10163000553029F4B991A991B095A09545C056307F
:1016400009F4E3C1573009F493C2583009F4CDC20C
:10165000593009F4E2C25A3009F4FDC25B3009F492
:1016600005C35C3009F406C35D3009F408C35E307D
:1016700009F4DEC2503109F410C2513109F42BC112
:10168000523109F42EC1533109F414C2543109F412
:1016900029C25F3009F444C3553109F4C2C156313F
:1016A00009F4D6C1573109F4DBC1583109F474C2C9
:1016B000593109F487C2503029F06ED0803009F0DA
:1016C00056C0A4CF86E00895AA93BA93AA27BB2751
:1016D00042E0D8CE4F3720F44F3010F086E047C0BC
:1016E0007C3361F471E260816E3319F472E26191CE
:1016F00042C06D3311F473E261913DC07E3339F421
:1017000074E260816D3311F475E2619134C07D3310
:1017100011F476E230C07B3211F470E32CC07D32DC
:1017200011F471E328C0733211F472E324C07A32E9
:1017300011F470E420C07F3211F471E41CC07532E2
:1017400011F472E418C0763211F473E414C05F919E
:10175000503021F05F3130F01FD0F9CFB991A9910D
:101760003197089586E05F915030C1F3FCCF4F91DF
:101770004030E9F708955F91A72FB52FA07FB07F84
:10178000BA1720F009D0803091F7F5CF5F937F939F
:10179000AA27BB27472F76CE5F934F9319910991C4
:1017A000B991A991513211F4FED03AC0523221F4CC
:1017B000F3D0A150A17034C0533221F4FCD0A15019
:1017C000A1702EC0543211F4F6D02AC0553221F443
:1017D000EAD0A150A17024C0563211F4DDD020C04F
:1017E000503311F441D01CC0513311F43CD018C017
:1017F000523319F4A02BB12B13C0503411F43FD045
:101800000FC0513411F4A7D00BC0523421F4A3D02F
:10181000A22FB32F05C0533419F4A023B12300C065
:10182000AA93BA934F915F910895B991A99103D06A
:10183000AA93BA930895B7FF0895A095B095A30D04
:10184000B21D089517FF089500951095030D121D00
:101850000895B991A991AB2B29F0B7FBA1E0BB2763
:101860000EF41297E5CFF0DF2B2F2127A00FB11F29
:1018700027FD08952B2F212727FD82E008950CD006
:10188000A22FB32FBF770EF4D8DF37FD03C0452B4F
:1018900009F4089582E008957AD0CDDFB19F402DFC
:1018A000512DA09F202D312DA19F300D411D521D86
:1018B000B09F300D411D521D089508E611E0B0386B
:1018C00018F0A00FB11FFBCFA017B10718F0A01B95
:1018D000B10BFACF0895B991A9910AE5A01BB209FD
:1018E00002C0B991A991E9DFFF93EF93E0EAF1E833
:1018F0000AE510E0A017B10748F4E00FF11FEA1B5A
:10190000FB0BA491EF91FF91BB27DECE04EB10E01F
:10191000A017B10778F40AE510E0E01BF10BEA0F1D
:10192000FB1FA491EF91FF91BB27A095B095A30D4C
:10193000B21DCACE0EE011E0A017B10728F4E00FE7
:10194000F11FEA1BFB0BEDCF0EE011E0E01BF10BEA
:10195000EA0FFB1FD6CF212F202B11F483E008952F
:1019600016D022273327442751E1441FAA1FBB1F4B
:101970005A9551F0221F331F4FEF201B310BA8F750
:10198000200F311F40E0F1CF0EF457CF08952B2FD9
:10199000212727FB50DF56CF0A271B27AA27BB2763
:1019A000012B89F00895B0581058A01BB10BAA273D
:1019B000BB2748F00895B05810580A1B1B0BAA27E4
:1019C000BB2708F00895A1E0B0E00895B991A9916E
:1019D00084E0B7FD08950F931F932F933F938827BB
:1019E0000A2F1B2FB2E0AA27232D3327021B130B2C
:1019F00020F0A3952B0F321DF9CFBB27AA93BA93E2
:101A00003F912F911F910F9108954F935F930E94E3
:101A100067381991099142DFA42FB52F5F914F913B
:101A200053CE19910991023039F420925801A2E065
:101A3000A0933B01BB2748CE013031F4A0913B017C
:101A4000A03011F430923B01A0913B01BB273CCE6A
:101A5000199109910EBD0E94E419AEB5BB2734CE91
:101A600010914601103011F08CE1089519910991FF
:101A7000A4ECB2E00A171B0710F082E10895FF936F
:101A8000EF93FDE0ECE3E00FF11F68940E94F23762
:101A9000EF91FF91A42FBB2717CEB991B0937F018F
:101AA000A991A0937E01CF93DF930E94E819DF9163
:101AB000CF910ACEB991A991BF3F71F0A093640173
:101AC0000E948A22803021F0AFEFBFEF8827FCCD43
:101AD000A42FBB270C94640B0E948F228827B42F5D
:101AE000AA27F2CDB991A991BF3F21F5A0FD11C060
:101AF000DF93CF93FF93EF930E948722803019F0FA
:101B00008827CC27DD27DE01EF91FF91CF91DF9170
:101B1000DBCDDF93CF93FF93EF930E94872280303A
:101B200019F08827EE27FF27DF01EF91FF91CF9172
:101B3000DF91CACDA09364010E948A22803021F0F7
:101B40008827AA27BB27C0CDDF93CF937F93772722
:101B50000E949222DF3F41F4CF3F31F4A72FBB27F1
:101B60007F91CF91DF91B0CD7395703889F7F6CF23
:101B7000A991A991A770A06CA0937C00A0917A0074
:101B8000A064A0937A00A0917A00A6FDFCCFA0915A
:101B90007800B091790098CDB991A991BB3020F42B
:101BA000BA3028F0A83C18F0AFEFBFEF8DCDEF931F
:101BB000FF93E4EDF1E0EA0FFB1FA081BB27FF914B
:101BC000EF9182CDB33018F4B23010F0A7FDCFCD35
:101BD000DF93CF93CCE3DDE0CA0FDB1F0E94AD3C67
:101BE000A62FBB27CF91DF916FCDB991A991B030CE
:101BF00061F4AF3F79F0A770A395B0B1B695AA95FF
:101C0000E9F7AA27AA1FBB275FCDBA2FA0B1AB2344
:101C1000BB275ACDA0B1BB2757CDB991A9910E943E
:101C20001A790E94233D8030E9F4BB27A52F4CCDC3
:101C3000B991A991CF93DF93CA2FDB2F0E94633D07
:101C4000DF91CF91803019F4BB27A42F3DCDAA2777
:101C5000BB2782E288CDA99179910E94413D8030D5
:101C600009F432CDAA27BB278FE07DCDB991A99188
:101C7000BB272ACDB991A991AB2FBB2725CD0F93B7
:101C8000B9910991AA27BB27003019F4A0911E0130
:101C900045C0013029F4A0911E01A030E1F33EC0FF
:101CA000023039F4A0911E01A030E1F7A0911F018C
:101CB00035C0033019F4A0911C0130C0043039F450
:101CC00000911C0100FD119602FD119727C00530FF
:101CD00039F400911C0101FD119603FD11971EC0FE
:101CE000063049F400911E01023E09F41197033EAB
:101CF000A9F4119613C0073049F400911E01043E67
:101D000009F41196053E51F4119708C01F931091E4
:101D10001E010117E1F71F91A02FBB270F91D4CC13
:101D2000B991A991BB27A13021F4A0917901A39584
:101D3000CBCCA23021F4A0917A01A395C5CCA0917F
:101D40007B01C2CC4142532053474E205351522075
:101D50004E4F5420524E442041444320494E205877
:101D60005045454B2054454D50204C4F204849206C
:101D70004B455920455045454B2045525220415234
:101D80002053494E20434F53204654595045204636
:101D900053495A45205053544154205350494D45BE
:101DA0004E552056425954452000FCE0ECE9A0E095
:101DB000B4EBA193BA95E9F7F1E0E4E7B0E1A193C0
:101DC000BA95E9F7FDE0ECE3B0E0A193A193A1930C
:101DD000BA95D9F7DD24CC24209217012092150161
:101DE000AEE0A0933401ACE3A0934C01AEE2A0932B
:101DF0004D01AFEFA0938301A093080120920B0146
:101E00000E94A13120925801A2E0A0933B01A6ECD0
:101E1000A0937A00409145014093420140933F01D5
:101E20000E9424799C2D0E94407921D0803039F481
:101E3000AC2DAF35B8F39CE0209258010895C092C4
:101E40007901D0927A0180937B01813051F0209208
:101E50005801409183014F3520F4DD24C42E88279A
:101E6000E1CF9CE0209258010895F7012AC0F1E0EB
:101E7000ECEA209232018827AD2DBB27AB1709F180
:101E800071917F3FD1F07C31D1F07E31C1F07D3155
:101E9000A9F07F3199F0773281F0723241F471917B
:101EA0007F3F59F0773249F07232C9F7E9CF7A3380
:101EB00039F7B395AB1721F704C02FC07191719119
:101EC000DFCF7091350170FF05C081E07E7F709398
:101ED0003501089572FF11C0AB7F70933501A09159
:101EE0004601A53011F0A03011F40E94E11CA0FFC2
:101EF00004C00F900F9081E008950E94F136709118
:101F00000B01703039F0A0910801DA9420920B0196
:101F10000C94581371917F3F19F4DD24C3940895F4
:101F200077FD2BC0703269F27A3311F4D394C9CFA4
:101F3000773219F27134D8F07B3528F07052713451
:101F4000B0F07B35A0F4672E0E9474187D3379F4CD
:101F500090DA803069F4762D7154770FDCE0CCE9AB
:101F6000C70FD21DA993B99381CFEF91FF9187E05D
:101F70000895703810F487E078CF7F01E5ECF72FF3
:101F8000FF73EF0FFFE0F21D099449C0F3C0D2C206
:101F900068C13EC125C36DC37BC775C376C37AC311
:101FA0003AC0C8C6E6C67AC3E4C308C33CC46CC41E
:101FB000AAC1AEC4BEC4C3C41BC2C7C2C8C4D3C4B2
:101FC000DAC492C57CC107C1A9C25DC11AC5DDC40E
:101FD00024C01BC53CC580C215C3FFC5F1C751C68F
:101FE0005DC662C6A5C1E4C635C7C2C763C672C6B0
:101FF0008CC24DC594C651C1B3C2D9C33FC3D5C469
:10200000D7C46FC1A7C176C6C4C188E0089584E172
:10201000089583E108950C9426190C9440190E94A8
:1020200078189CE0732C20923201B191B032E9F320
:10203000BA3321F0B73211F0BF3F59F4319770FC39
:102040000E94DF3140913201443010F00E94ED3C9B
:102050000DCFBB3311F47724E8CFBC3291F440911B
:102060003201403031F40E940F32BA2DB770D9F7E7
:1020700006C00E940F32B0913301B770D1F77724B8
:10208000D4CF732CB332C9F420926401209265013D
:10209000F0D94A2F40933201443018F4433001F410
:1020A000C4CF0E94F13C683051F5509132015E7FFF
:1020B0000E94F33C683119F5B8CFB03411F5E3D77D
:1020C00040913201433018F40E94BB33AECF39F453
:1020D000A0936401B0936501A0933301A6CF5FEF95
:1020E0000E94F33C683259F45A2F0E94F33C683244
:1020F00031F45B2F0E94F33C683209F496CF8FE0F5
:102100000895B13229F4B5D99A2F8FCF97CF8DCFBB
:10211000B23241F441914F3FC9F34232C1F30E94C0
:102120001032F8CFB63291F4A4D9B33010F082E176
:102130000895CCE3DDE0CA0FDB1F4991403029F060
:102140000E9410321196B330C0F36FCFB53229F42C
:1021500090D94A2F0E94103268CF31978AD98030A7
:1021600009F00895903818F40E9431315ECF0E9432
:102170008C315BCF703CB8F4A1E037D7B091460109
:10218000B63019F00E94A13170CEA13029F00E9422
:10219000C8380E94D43869CEB0916401B130C9F317
:1021A0000E94C83862CEA2E020D7A23081F5A0E814
:1021B000B2E060916401C0916601D0916801CA17D4
:1021C000DB0738F4ACE3BDE0CA0FDB1F0E94D03C54
:1021D0004CCE82E10895A2E008D7A030C1F0A13032
:1021E00059F0A0916601A770AA0FB0913401B770A1
:1021F000A295BA2BB0933401A0916401A770AA0FE5
:10220000B0913401B07FBA2BB09334012ECE01CF00
:10221000A3E0EBD6A33018F1A0916401B091650161
:10222000A0937E01B0937F01A0916601B0916701F8
:10223000A0936401B0936501A0916801B091690118
:10224000B03011F4A03051F00D010E94E8190E9445
:10225000CD18D001803021F41197F2CF06CED9CE1F
:102260000895A5E0C2D6A43068F0CED77F93FAD601
:10227000E0937701F09378010E94F4347F9170939A
:102280003401F3CDC6CEA1E0B0D6A130D8F3409151
:102290006401417040931501E8CDA5E0A6D6A430B5
:1022A00068F0B2D77F93DED6E0937701F0937801A0
:1022B0000E9416357F9170933401D7CDAACEA5E048
:1022C00094D6A43068F0A0D77F93CCD6C093770182
:1022D000D09378010E94373A7F9170933401C5CD35
:1022E00098CEA5E082D6A43068F08ED77F93BAD678
:1022F000C0937701D09378010E947E3A7F917093CA
:102300003401B3CD86CEA3E070D6A23080F07CD766
:102310007F93B0916401A0916601A0937701B0937F
:1023200078010E94CE337F91709334019ECD71CE9F
:10233000A5E05BD6A43068F067D77F9393D6E0938F
:102340007701F09378010E94D0357F91709334012A
:102350008CCD5FCEA0914601A03011F08CE10895A4
:10236000A1E043D6A130A8F3A0916401B09165012A
:10237000CCE3DDE0CA0FDB1F409134014F93AF92F5
:10238000BF920E94C13ABF90AF904F9140933401E9
:102390006CCDA0914601A03011F08CE108958DD64E
:1023A000C0937E01D0937F019FD67C32F9F4A1E0E7
:1023B0001DD6A13070F2A0916401B0916501CCE30B
:1023C000DDE0CA0FDB1F409134014F93AF92BF9203
:1023D0000E94EA3ABF90AF90C0917E01D0917F01F8
:1023E000499329924F91409334013FCD87E03DCDF1
:1023F000A0914601A03011F08CE108955ED6C09303
:102400007E01D0937F0170D67C3281F7A1E0EED5BA
:10241000A13009F0FECDFF93EF93AF92BF924091B0
:1024200034014F937F934F70409334010E94A51B5A
:10243000C1E0D2E0ECE1F5E10E946A35C0913401DF
:10244000C295C09334010E94A23303020000A09100
:102450006401B0916501CCE3DDE0CA0FDB1FA6E1AA
:102460004991403230F0403820F40E941032AA9551
:10247000B9F7772761E025D00E94C71B623079F455
:10248000C0917E01D0917F01799329927F914F91E4
:1024900040933401BF90AF90EF91FF91E6CC7F91D4
:1024A0004F9140933401BF90AF90EF91FF91C09155
:1024B0007E01D0917F014FEF49934993D6CC87E0BD
:1024C000D4CC0E9418198827603009F408950E941E
:1024D0003320882762E00895A3E087D5A230A0F0DA
:1024E00093D67F93D0917801C0917701F0916401E8
:1024F000E0916601E0937701F09378010E94D03576
:102500007F9170933401B1CC84CDA4E06ED5A4301A
:1025100021F4A8D50E94CC34A8CC7BCDA1E065D510
:10252000A13090F0A0916401A295AA0FAF7EA09374
:1025300017019BCCA1E059D5A13030F0A0916401E6
:10254000A150CA2EDD24089564CDA1E04ED5A1305E
:1025500030F0A0916401A150A093830186CC59CDA5
:10256000A5E043D5A23040F1F0916401F770E0E0BE
:10257000EF0FF1E0B0916601B770BB0FB295B19368
:10258000A230C9F0E770B0916801B770BB0FB29587
:10259000B193A33081F0E770B0916A01B770BB0FBF
:1025A000B295B193A43039F0E770B0916C01B77077
:1025B000BB0FB295B19359CC2CCD2BCDA1E015D545
:1025C000A130D8F3A0916401A770A73041F00E9418
:1025D0009E30A0914601A63010F40E94A13145CC56
:1025E000A1E003D5A13068F0A0916401B09165012C
:1025F000B03019F4A03009F438CC0E940536119798
:10260000F7CF07CD20925801A2E0A0933B01A3E0B1
:10261000ECD4A33058F1CCE3DDE0A0916401B0919B
:102620006501B33020F5AC0FBD1FA0935A01A093F4
:102630005C01B0935B01B0935D01AC1BBD0B0090DE
:1026400066010A94A00DB21DA00DB21DB33078F43E
:10265000AC0FBD1FA0935E01B0935F01A091680114
:10266000A09358013092600120923B01FECB82E1A1
:10267000FCCB20925801BF91BF9108953BD5AB2B65
:1026800009F41BCCF3CB34D5F1CBF701FCD40E9479
:10269000BB33ECCB2FD50E940E36E8CBA2E0A5D4FD
:1026A000A13019F0A23021F1B4CCA0916401AA9517
:1026B000AF3510F08AE0D9CBB0917C01BC3010F07E
:1026C0008DE0D3CBAF93C8EFDCE0A5E0AB9FC00DAE
:1026D000D11DB395B0937C01BD2DB395B068B9936E
:1026E000BC2DB993B0914501B993DD24CF900895E5
:1026F000409164014A950E94B9794E3469F4A091E1
:102700006601B0916701B630A8F6F695E795EA0F35
:10271000FB1F38960995A9CBA0916601AA95AF3504
:1027200048F6B0916401BA95B770B0933F01B0918B
:102730007C01BC3010F08DE098CBAF93C8EFDCE0AB
:10274000A5E0AB9FC00DD11DB395B0937C01BD2D0D
:10275000B395B068B993BC2DB993B0914201B993C8
:10276000DD24CF9040913F01409342010E942479A3
:102770000895BED4B0917C01B03011F48CE008957E
:10278000BA95C8EFDCE0A5E0AB9FC00DD11DB093BA
:102790007C01B991B7FFF2CFBF77DB2EC990499189
:1027A000409342010E942479089587E00895A0D4BF
:1027B0009BD47134D0F37B35C0F77154770F672EFB
:1027C00093D47D3391F70E94390A803009F008953F
:1027D000DCE0CCE9C60DD21DA993B99385D474353C
:1027E00021F771917F3409F70E94390A4A2E5B2E36
:1027F000803009F00895B0917C01BC3010F08EE07B
:102800000895C8EFDCE0A5E0AB9FC00DD11DB395E6
:10281000B0937C01BD2DB395B993BC2DB99369924A
:102820004992599223CB64D4B0917C01B03011F419
:102830008BE00895BA95C8EFDCE0A5E0AB9FC00D32
:10284000D11DB991B7FDF4CFBF77B0937601599000
:102850007991BCE0ACE9A70FB21D0D911D91030D5C
:10286000121D1E930E93A991B99111960A1741F466
:102870001B1731F4B0917C01BA95B0937C01F6CA74
:10288000C52CD09076010895A0914601A03011F09A
:102890008CE108952DD4BFEFB0938401B191B03293
:1028A000E9F34B2FBF3F21F40E94DF313197DECA9D
:1028B000BA33D1F3BB3391F3BC3231F40E940F32FF
:1028C000BA2DB770D9F7EACFB23241F441914F3FF8
:1028D00059F3423219F30E941032F8CFB134B0F0FC
:1028E000BB35A0F4B154BB0FB0937601B081B134C5
:1028F00018F0BB3508F40AC000D4DCE0CCE9109134
:102900007601C10FD21DA993B993C8CF87E008956E
:10291000F1D3803009F0AACA4A2F4B2BE1F3409142
:102920002A014030E1F340912A014030E1F711974C
:10293000F3CFE0D3A0932B01B0932C01EDCFBDD307
:10294000A0912B01A993A0912C01A9938FCAD2D356
:102950004A2F0E94BF37C9D37C3221F4C5D30E94CD
:10296000390AF6CF83CA0E94CB37A42FBB27A5D341
:10297000A993B9937BCAF70193D34A2FD73020F498
:10298000C03D10F40E946C3D71CAF70189D35A2FE3
:10299000AC2FBD2F0E941A790E94363D0E94053649
:1029A0000E9405360E94053661CAA4D3A1B95ECA49
:1029B000F70176D3D030B1F4BC2FB770B395772739
:1029C0006FE7A0FD70E8A0FD6FEF77FB770F70F960
:1029D00067FB660F60F9BA95C1F702B1072B0623B2
:1029E00002B944CAD13041F4B2B1C095BC23C095FC
:1029F000CA23BC2BB2B93ACAD230E9F70E94D21925
:102A000035CA78D30E94AB3731CA57D3C0937E0101
:102A1000D0937F0109911991105866D37C32A9F4A3
:102A20003FD3B058D058C017D10710F00C2F1D2F2E
:102A3000A017B10710F40A2F1B2FD0917F01C0916E
:102A40007E0110580993199311CA86E00895A09148
:102A50004601A03011F08CE108952FD3C0937E0180
:102A6000D0937F0141D37C3281F70DD3C4EDD1E007
:102A70007EE17B9FC00DD11DCA0FD21DBB27A8814F
:102A8000D0917F01C0917E01A993B993EFC9A09124
:102A90004601A03011F08CE108950FD3C0937E0160
:102AA000D0937F0121D37C3281F6EDD2C4EDD1E009
:102AB0007EE17B9FC00DD11DCA0FD21DA2EBCA0FB4
:102AC000A2E0DA0FBB27A881A695BA2FA777B29507
:102AD000B078AB2BBB27D0917F01C0917E01A99329
:102AE000B993C4C986E00895E8D2C0937E01D0931B
:102AF0007F01FAD27C32B1F7C6D2C4EDD1E0709139
:102B000046017770703021F5AF93BF93A695B695C7
:102B10007EE17B9FC00DD11DCA0FD21D7881BF9170
:102B2000AF91A0FD7695B0FD7695B0FD7695A2EBC0
:102B3000B2E0CA0FDB1FA88170FFA295A695A7700F
:102B4000BB27D0917F01C0917E01A993B9938EC913
:102B50007130B9F4AF93A695A695A69575E17B9FC4
:102B6000C00DD11DCA0FD21D7881AF91A2FD729503
:102B7000A1FD7695A1FD7695A0FD76957170A72FA4
:102B8000DECF7230A1F4AF93A695A6957EE17B9F30
:102B9000C00DD11DCA0FD21D7881AF91A1FD7295D4
:102BA000A0FD7695A0FD76957370A72FC8CF7330E2
:102BB00071F4AF93A6957AE27B9FC00DD11DCA0F29
:102BC000D21D7881AF91A0FF7295A72FB8CFAF9398
:102BD000A695A695A69570E1C2CFA0914601A0301A
:102BE00011F08CE10895A3E000D2A33080F0A09111
:102BF0006401B0916501B33010F082E10895B23004
:102C000039F4A73F28F082E1089581E2089501CACE
:102C1000CCE3DDE0CA0FDB1FC0934E01D09351011E
:102C2000AC81A03091F3AE3180F7BB81B03069F355
:102C3000B73158F7C0916401D09165012596BA9FCC
:102C4000000C111C000C111CC00DC11DD330E8F686
:102C5000D0916601C0916801C0935001D093530197
:102C6000CF3F51F0DF3F41F0CA0FCA95CE3138F463
:102C7000DB0FDA95D73118F40E945C3BF6C886E189
:102C80000895A0914601A03011F08CE1089530D252
:102C9000A0913501A460A0933501E8C8A09131014D
:102CA000A062A0933101E2C8A0913101AF7DA09351
:102CB0003101DCC8A3E099D1A33009F0AAC90E9470
:102CC0008A22403310F08EE108950E949E228030C7
:102CD000D9F7CBC8A3E089D1A33009F09AC90E94E3
:102CE0008A22403310F08EE108950E94A1228030A4
:102CF000D9F7BBC8A3E079D1A23019F0A33021F0F5
:102D000088C9A4E1A09368010E949822803009F448
:102D1000ACC808950E949B22803059F4A6C8A1E057
:102D200064D1A13009F075C90E948A22443191F31F
:102D30008EE10895A2E059D1A23009F06AC9A091AC
:102D40006401B091650140916601CCE3DDE0403063
:102D500041F0D395413029F0D395423011F082E112
:102D600008950E94CC3D0E94BC3E803009F0089539
:102D70007CC8A2E03AD1A23009F04BC9A09164010D
:102D8000B091650140916601CCE3DDE0403041F057
:102D9000D395413029F0D395423011F082E1089566
:102DA0000E94863E0E94E83D803011F308954EC097
:102DB000F7014DD1A09380010E94F13C6830B9F732
:102DC00090FF28C0592F0E94F33C603481F7A03057
:102DD000C9F0DDE0CCE3409180014B0F4A1BC40FEA
:102DE000D21DA13039F00E94F73C603579F5588347
:102DF000AA95EFCF0E94FC3C683541F558830E94AC
:102E0000ED3C34C80E94F73C5030A1F35093800150
:102E1000A52FDFCF592F0E94F33C6831B9F43A2F28
:102E2000DDE0CCE3409180014B0F4A1BC40FD21D63
:102E30005881503011F4303031F00E94F33C683248
:102E400029F4AA9569F70E94ED3C10C88FE00E9412
:102E5000ED3C08954FD1A0936401B093650145D135
:102E60007C3249F4319640D1723239F031970E9468
:102E7000390A93D1F4CF0C94360F7191723231F03C
:102E80007F3F21F0BB27A72F88D1F7CF7081E7CFF5
:102E9000A0914601A03011F48DE10895A43011F005
:102EA000A63028F0A2D0A43079F40C945A19A7E0E7
:102EB0009CD0B0916401B0935401B13039F0B2307C
:102EC00011F1B33009F43DC085E10895A730E1F771
:102ED000C4E6D1E0BA81B0935101BC81B0934E01F8
:102EE000BE81B0935201B885B0934F01BA85B093BB
:102EF0005301BC85B09350010E94E338803009F043
:102F000008950C94350FA630F9F6C4E6D1E0BA81E5
:102F1000B0935101BC81B0934E01BE81B093520178
:102F2000B885B0934F01BA85B0935001BB85B0937B
:102F300053010E94E338803009F008950C94350F56
:102F4000C3CFA430E9F7C4E6D1E0BA81B0934E0113
:102F5000BB81B0935101BC81B0935301BE81B0934A
:102F600050010E94E338803009F008950C94350F29
:102F7000A0914601A03011F08CE10895F70190D0A6
:102F8000C0936401D093650150918001A51708F4A6
:102F90005A2FA4E8B1E0503071F04D91A093810117
:102FA000B0938201A42FBB27F8D0A0918101B091EA
:102FB00082015A95F0CFAA27BB27EFD00C94360F89
:102FC000A0914601A03021F0A43011F08CE10895C9
:102FD000A1E00BD0A13040F0A09164014A2F4370D2
:102FE0000E94213C0C94350F14C8F701A03009F45D
:102FF0000895DF93CF93C4E6D1E040E05A2F5030DC
:1030000029F4A42F7F01CF91DF910895DF93CF930F
:103010004F935F930E94390A5F914F91CF91DF9157
:10302000893121F488277F01A42F0895A993B993AA
:1030300043955A95503019F371917032E9F37C320F
:1030400029F33197A42F7F01CF91DF910895A3E059
:10305000CCDFA33009F590916401B0916601A09195
:1030600068010895D0916401C0916601F0916801F2
:10307000E0916A01C0934E01D0935101E0934F015A
:10308000F09352010895A2E0B1DFA23029F4B0918B
:103090006401A09166010895AF91AF910C9409105D
:1030A000A2E0A4DFA230C1F7C0916401D091650114
:1030B000A0916601B09167010895F70115D07134B0
:1030C00078F07B3538F47154770FDCE0CCE9C70F2A
:1030D000D21D0895713620F07B3710F47156F4CF6D
:1030E0008F918F9187E0089571917032E9F308957F
:1030F000F7010895F7010C94390AEF93FF930E94AA
:103100009A36EC2FFD2F00E00E943A36709135017F
:10311000713011F4872F08C04A3EC9F40093800132
:10312000003031F4AA27BB278827FF91EF9108953B
:10313000C4E8D1E0A191A9930A95E1F7A0E2A9938F
:10314000AFEFA993E4E8F1E00E94390AEDCF4C3EDD
:1031500049F40030C9F2AA940E949A36A0E2A883EA
:103160000A95D2CF403248F24B3738F6AA2DAD310E
:1031700020F60E9410320395C7CF92E0BB27AC2DFA
:10318000A3950E9431314AE30E941032BB27AD2D36
:103190000E9431310E940F320895DF93CF93BF9385
:1031A000AF93A0916401B0916501B33098F4CCE382
:1031B000DDE0CA0FDB1FAF91BF91A883C09164010E
:1031C000D09165012196C0936401D0936501CF91A0
:1031D000DF910895B45090F0AA0FBB1FB33070F484
:1031E000CCE3DDE0CA0FDB1FAF91BF91A993B99388
:1031F000C0916401D09165012296E5CF82E1AF9143
:10320000BF91CF91DF91089570913401A0FF08958F
:10321000A33059F4509168015F70550F707F572BA0
:103220007091340150933401089550916C01F4CFA2
:103230000E94A422403011F46627089540936C0147
:103240000E949522413009F066270895A2E0CDDE64
:10325000A130A0F0B1E0A13011F0B0916601A091D1
:103260006401A150A0930801B09309010E940536A2
:10327000B0930A0120920B010C94350F0C940910A5
:10328000A2E0B3DEA230D0F3C0916401D091650119
:10329000DB3020F4DA3028F0C83C18F086E10C94DA
:1032A000350FA4EDB1E0CA0FDB1FA0916601A88322
:1032B0000C94350FFF93EF930CE310E12CE93CE005
:1032C000B0916401B13019F5E4EDF1E0A09166012F
:1032D000B0916701BF70AE0FBF1FC0916801D09160
:1032E0006901DF70CE0FDF1FE0916A01F0916B0181
:1032F000A217B30740F4C217D30728F4319718F088
:103300000D900992F5CFEF91FF910C94350FB230EB
:1033100009F5E4EDF1E0A0916601B0916701BF709D
:10332000AE0FBF1FECE3FDE0C0916801D0916901D1
:10333000DF70CE0FDF1FE0916A01F0916B01A217E1
:10334000B30708F7C017D107F0F63197E0F20D90F8
:103350000992F5CFB33011F5ECE3FDE0A0916601E1
:10336000B0916701BF70AE0FBF1FE4EDF1E0C091F7
:103370006801D0916901DF70CE0FDF1FE0916A0113
:10338000F0916B01A017B10740F4C217D30728F4DE
:10339000319718F00D900992F5CFB5CFEF91FF91CD
:1033A00085E10895AF3F31F42C9A2CBCACE5ACBD5F
:1033B0003DBC0895A7F92CBCAF73A064ACBD3DBC67
:1033C000A5B1A4FBA5B90895BDB5B7FFFDCF08957C
:1033D00050917E0140917F01433038F4DDE0CCE331
:1033E000C50FD41FA991BB2710C05050444058F0BE
:1033F000550F441F433038F4DDE0CCE3C50FD41F34
:10340000A991B99102C082E1089540917E01509145
:103410007F01430D521D40937E0150937F01803008
:1034200009F408954F914F910895ACEAB1E04FEF40
:1034300052E24D935A95E9F7C4EAD1E040E25A913D
:10344000503211F44A95D9F7442EACEAB1E0C4E801
:10345000D1E04C0EAC3C28F4C41518F4488140303F
:1034600009F408958BD04F3FE1F372D04F3FC9F379
:10347000403081F790D0403069F73DD0403051F76F
:103480000AD0403039F74991413618F04B3708F4EB
:1034900040524D93DFCF4881403320F04A3310F43F
:1034A000405302C044270895642F7727219648810E
:1034B000403380F04A3370F44053660F771F0B019E
:1034C000660F771F660F771F600D711D640F721DE9
:1034D0002196EDCF703029F04DE14D937D936D93A2
:1034E00008956A3020F04CE14D936D930895605D2E
:1034F0006D934CE108954881443211F044270895BA
:1035000066277727219658815033B8F05A3328F42C
:10351000505309C05A3508F05052513470F05734A6
:1035200060F4575300C05F70529544E0550F661F1A
:10353000771F4A95D9F72196E6CF703029F04FE1F1
:103540004D937D936D9308954EE14D936D93089542
:103550004881423211F04427089521964D934991B4
:10356000423219F44D9341E00895403029F442E28B
:103570004D934FEF4D9308954D93F1CF48814732CE
:1035800011F04427089521964D9349914030E1F779
:103590004FEF4D930895FF93EF93BF93AF935F93D6
:1035A000EAE8FBE40E014591403089F0689457E069
:1035B000A591AE3239F0B991B13608F0B052AB17DF
:1035C00009F0E8945A95A1F716F0E001EBCF5F916E
:1035D000AF91BF91EF91FF91403041F04D934F93E8
:1035E0004881403211F42196FBCF4F910895C7E8EE
:1035F000D1E0ACEAB1E040E2E0E24993EA95E9F7D4
:10360000A097AC3C29F04D91423010F04F3F11F49F
:1036100029920895403220F0403810F486D0F1CF3E
:103620004C3121F4ED91FF2719D0EBCF4D3121F42E
:10363000FD91ED9113D0E5CF4E3131F444E275D0D8
:10364000ED91FF273CD0DDCF4F3131F444E26DD016
:10365000FD91ED9134D0D5CF50D0D3CFE8944FE247
:103660004395E051F742E0F7E05FF84D403311F049
:1036700063D068944FE24395E85EF340E0F7E85189
:10368000FC4F16F0403311F057D068944FE2439549
:10369000E456F040E0F7EC59FF4F16F0403311F0DC
:1036A0004BD068944FE24395EA50E8F7E65F16F096
:1036B000403309F041D040E34E0F3ED00895E894E6
:1036C0004F2F42954F7011F012D068944F2F4F70CA
:1036D0000EF011F00CD068944E2F42954F700EF002
:1036E00011F005D068944E2F4F7001D00895405DC1
:1036F0004A3308F0495F20D00895EAE8FBE4559189
:10370000503009F40895451711F03796F8CF5F93BC
:1037100057E045914E3209F00FD05A95D1F75F919D
:103720005C3110F040E208D008954993C73A18F090
:1037300029924F914F9108954993C73A28F02992C1
:103740004F914F914F914F910895A0914601A093B1
:103750007A01AA270E949E30A0913401A09376019D
:10376000A0911701A0937901A0913201A093750156
:1037700020923201E4EDF1E0C8E3D7E0BEE2AEE131
:1037800041914993AA95E1F7BA95C9F70895A09197
:103790007A010E949E30A0917901A0931701A09117
:1037A0007601A0933401A0917501A0933201E8E362
:1037B000F7E0C4EDD1E0E2CFC2E1D4E0E4ECF6E022
:1037C00041B150B168E0A9E4BFEA469510F4AFE416
:1037D000BFE2A993B193A0E3B0E8569510F4A1E33A
:1037E000BEE4AD8FB58F6A9571F70895452FA6E1B8
:1037F0000E9409314F5B0E9410324DE30E9410324B
:10380000A7E10E940931CCE9DCE0C50FD21DC50F4C
:10381000D21DA991B9919DE00E9431310895A3E193
:103820000E94BB33A5E0C62FCA95AC9FC8EFDCE071
:10383000C00DD11DA881A7FF09C00E94A233FF437C
:10384000414C4C202000A981AF770DC00E94A233CB
:10385000FF464F5220004A8146954F5B0E9410322E
:103860000E940F32A981BB27A39592E00E943131BB
:103870004AE30E941032BB27A881AF770E94313102
:103880000895209217019927A7E00E9409310E940C
:10389000A1310E94A2331200424954203031323308
:1038A0003435363700000E94A233130044495200D9
:1038B0000E94A23314004C455600ECE9FBE30E9441
:1038C0004538A5E00E9409310E94A233000041560C
:1038D000522D43686970426173696332204D4F4EC7
:1038E00020202020500040913F014F5C0E94103268
:1038F0000E94A233FF3A000092E0BB27AC2DA395B3
:103900000E9431310E94A233FF3A0000BB27AD2D47
:10391000A3950E943131E7E8F1E0C2EFD1E0AEE1DA
:1039200041EFB191B03031F0BE8F4CAF4993AA95C1
:10393000C1F706C0B0E2BE8F4CAF4993AA95D1F74C
:10394000A7E10E940931C0E0D4E0E1E1F0E10E948A
:10395000CC349DE050E0452F4C5FB42FAA270E9445
:10396000BB3344DF53955D30B1F7452F4950B42F39
:10397000A9E00E94BB333ADF53955A31B1F7A7E370
:103980000E940931C3E1D4E0EDE1F0E10E94CC34C2
:103990000E94A2330413535441434B3A0000992729
:1039A000BB27A0917C010E9431316CE0C0917C0169
:1039B000C61720F0C61BB4E0B60F31DF6A95B1F729
:1039C00008954F935F936F937F93EF93FF93CF93FC
:1039D000DF93AF93BF93AF92BF928F939F93B5DE68
:1039E00006DE4FDF31D08827A09135014D3E11F41E
:1039F000A16014C0413F11F4AA2710C0423F11F446
:103A0000A4600CC0433F39F4C2DE0E942E36AA27C0
:103A10000E949E30E6CF443F29F71FC0A093350196
:103A200040911E014030E1F7B2DE9F918F91BF902F
:103A3000AF90BF91AF91DF91CF91FF91EF917F91C7
:103A40006F915F914F91089520921F01B5DE4091D3
:103A50001F014030D9F30C94F1360E94353670E0E6
:103A6000442425D0EEE7FBE30E9445380E942E3621
:103A70004D3E11F4A160D2CF443F19F40E94353677
:103A8000B0CF463E31F4703069F37A950E943536F6
:103A9000E8CF473E31F47A3028F773950E943536E7
:103AA000E0CF433FF9F643940E943536DACFA7E0E2
:103AB0000E9409310E94A1310E94A23300004156A8
:103AC000522D43686970426173696332204172729A
:103AD0006179205669657700A0E60E9409310E944D
:103AE000A2330200416472202000A0E50E94093147
:103AF0000E94A233020520202020202020202044E4
:103B0000617461202020202020202020202000001F
:103B100060E4679FCCE3DDE0C00DD11DF00163E000
:103B2000A0E0B62F0E94BB33A6E00E940931DF015E
:103B300091E00E948C31A5E0B62F0E94BB33A5E036
:103B40000E94093190E058E0A991B0E00E948C31C8
:103B5000442D40FF0BC0A7E10E94093121974991F4
:103B60000E941032A5E00E94093102C00E940F326B
:103B70005A9551F738966395633191F6089520452B
:103B80007869742020202020202020202020202040
:103B9000204368617220204D6F6E20202045786997
:103BA00074202020476F20202053746570202056F9
:103BB00069657720204172726179209232012092EA
:103BC0004601A5E00E940931C0E0D0E0EDE1F6E158
:103BD0000E946A35A0E50E9409310E94A2330102C9
:103BE00044464C4153482073697A653A20000E944C
:103BF000A4224F3749F40E94A233FF353132204BC3
:103C000069427974650011C04F3F41F40E94A233AC
:103C1000FF31204D69427974650007C00E94A233CC
:103C2000FF3020427974650013C00E949522413014
:103C3000D1F0E6E5FEE3E8940E94F237413009F462
:103C400034C0453009F4B9CF423099F733D0B5CFFD
:103C5000E2E9FEE3E8940E94F237413009F425C01E
:103C60004530B1F7AACFEAE1FEE3E8940E94F237CB
:103C7000413009F41AC0473019F40E94671F9DCFE4
:103C80004A3011F417D099CF423011F46DD095CF4E
:103C9000433019F40E94C01F90CF443019F40E94A1
:103CA00014208BCF4530F9F688CFA0911E01A030AB
:103CB000E1F708950E94DD3A4F466F726D617420FE
:103CC0004D656469756D3F00413009F00895A6E2C5
:103CD0000E940931C2E0D8E0EBE1FCE00E943235FD
:103CE0000E94A2330903466F726D617474696E6736
:103CF0002E2E2E202020202020000E94A2330B03F5
:103D000000000E94A722803001F50E94A23309031F
:103D1000466F726D617474696E672E2E2E20446F2B
:103D20006E652100A2E70E9409310E94A2330B03B5
:103D3000202020507265737320616E79206B657945
:103D4000212020000E942E3608950E94A2330903EC
:103D5000466F726D617474696E672E2E2E204572E7
:103D6000726F72210000DECFA0E60E940931C4E02C
:103D7000D8E0E9E1FDE00E9432350E94A233090556
:103D8000417661696C61626C653A00000E94A23301
:103D90000A0546696C65733A20009CE00E94872200
:103DA000DF93CF93DF010E9431310E94A233FF20C5
:103DB0002F000E94A422A42FB0E011960E9431315E
:103DC0000E94A2330B05426C6F636B733A00AF9194
:103DD000BF910E9431310E94A233FF202F000E9428
:103DE0008F22A0EFA49FD0011197B03009F4139750
:103DF0000E943131A6E00E9409310E94A2330C05D5
:103E0000202020507265737320616E79206B657974
:103E1000212020000E942E360895204578697420C4
:103E200020496E666F204261636B757052657374D2
:103E30006F7252657363616E2020202020204465DC
:103E40006C65746520202020202020202020202048
:103E5000466F726D6174204578697420466F726D8B
:103E60006174202020202020202020202020526546
:103E70007363616E2020202020202020202020201D
:103E80002020202020202020202020202020202032
:103E90002020204578697420202020202020202008
:103EA0002020202020202020202052657363616E76
:103EB0002020202020202020202020202020202002
:103EC0002020202020202020202020202020772794
:103ED0000FD1A4E00E940931C1E0D2E0ECE1F5E1AC
:103EE0000E946A35A0E40E9409310E94A2330302B5
:103EF00044656C6574652066696C6500B4D0709328
:103F0000640108D34C3FD1F350D1413019F4A72FAD
:103F1000C3D211D308957727EBD0A4E00E940931D2
:103F2000C1E0D2E0ECE1F5E10E946A35A0E40E9434
:103F30000931A0E1A09368010E94A23303025361FA
:103F4000766520500000CAD28ED070936401E2D210
:103F5000403E30F4403171F0483161F0F6D0DCCFB2
:103F6000D6D2D03021F4CC3010F429D1D5CF94D290
:103F7000B6D108950ED1413079F68ED2BCD10895D4
:103F80007727B6D0A4E00E940931C1E0D2E0ECE18D
:103F9000F5E10E946A35A0E40E940931A2E1A093F4
:103FA00068010E94A23303024261636B75700000D6
:103FB0005AD070936401AED2403920F4423161F09E
:103FC000C4D0DFCFA4D2D03021F4C03610F4F7D063
:103FD000D8CF62D226D20895DCD0413091F65CD29F
:103FE0002CD20895772784D0A4E00E940931C1E043
:103FF000D2E0ECE1F5E10E946A35A0E40E940931CB
:104000000E94A23303024C6F61642050000066D20C
:104010002AD0709364017ED2403121F0483111F0F2
:10402000A2D0E1CF90D10895772762D0A4E00E947A
:104030000931C1E0D2E0ECE1F6E10E946A35A0E48A
:104040000E9409310E94A2330302526573746F7299
:10405000650009D0709364015DD2423111F08ED0B9
:10406000E4CF03D208957727B5D00BD10E942E3626
:104070004D3E21F42FD14F914F9108954A3E09F4BE
:104080000895403E19F40FD17727EECF413E21F439
:104090000AD170916C01E8CF443E49F4703031F39D
:1040A00002D17150472F4F704F30F1F2DECF453EB5
:1040B00059F440916C01471709F4D8CFF4D07395A7
:1040C000472F4F7089F2D1CF463E29F4703170F2FC
:1040D000EAD07051C9CF473E51F440916C014F3046
:1040E00031F04051471718F0DED0705FBDCFBECF22
:1040F0000E94A422403019F44F914F911BC040936D
:104100006C010E9405360E9405360FD2413019F02D
:104110004F914F9101C008950E94B43A4F44464CCC
:10412000415348206E6F7420666F726D61747465C0
:10413000640008950E94B43A4F44464C41534820CD
:104140006572726F7221000008950E94B43A4F4365
:10415000616E206E6F742073617665206F6E2074BF
:104160006869730008950E94B43A4F4E6F2042412F
:104170005349432066696C65000008950E94B43A73
:104180004F4E6F204241434B55502066696C65008D
:1041900008950E94DD3AC04F766572777269746542
:1041A0002066696C653F000008950E94DD3A4F4427
:1041B000656C6574652066696C653F0008950E94B2
:1041C000B43A4F4E6F207370616365206C656674FE
:1041D000000008955F936F937F93A72FA07FA09314
:1041E0007801A0917801AF70AB5FBA2FA4E00E9474
:1041F000BB33A6E00E940931A0917801BB2795E06E
:104200000E9431310E940F32A5E00E940931A09135
:104210007801A09364017ED1B5D04F3F61F1A091A8
:104220007801A093640140E04093660142E040932E
:104230006801882783D1803091F4CCE3DFE00E94CD
:104240000F325CE05F934991403808F04EE2403213
:1042500008F440E20E9410325F915A9599F7A091BC
:104260007801A395A0937801AF7009F0BACF7F9140
:104270006F915F9108955DE00E940F325A95E1F7CA
:10428000EECF4F935F93C0E2D5E0472F4F705EE1D2
:10429000459FC00DD11D52EF47E159934A95E9F76B
:1042A0005F914F9108954F935F93C0E2D5E0472F00
:1042B0004F705EE1459FC00DD11D5CE044E0599315
:1042C0004A95E9F75AE043E159934A95E9F75F9136
:1042D0004F910895A0911E01A030E1F708957093C9
:1042E00064014CE04093660140E14093680120D1B5
:1042F000803009F01FCF7093640190914501ECE08C
:10430000F0E99770929540EC949FE00DF11D0491B7
:104310003C9740E10E3409F448E10E94FC3D40E046
:104320004F9300E0CCE3DFE0159119930A95E1F794
:104330004093660142E04093680103D14F91439559
:104340004C3071F70895909145019770E0E0F0E9E5
:10435000929540EC949FE00DF11D40E04F93409307
:10436000660142E04093680170936401E7D0CCE3BA
:10437000DFE00E947A7932964F9143954C3071F785
:1043800078940895403139F40E94A233FF4241539A
:104390003A0040E10895423139F40E94A233FF42CD
:1043A00055503A0042E10895443139F40E94A23355
:1043B000FF5553523A0044E10895463139F40E94C2
:1043C000A233FF4348383A0046E10895483139F4B2
:1043D0000E94A233FF42494E3A0048E108954A3113
:1043E00039F40E94A233FF47504F3A004AE1089542
:1043F0004C3139F40E94A233FF53414D3A004CE155
:1044000008954E3139F40E94A233FF4C424C3A00D9
:104410004EE108950E94A233FF2D2D2D2D004FEF68
:1044200008957093640140E64093660142E1409331
:1044300068017ED0803009F07DCE709364014427FE
:10444000E0E0F0E94F93CCE3DFE00024159019920F
:104450000A94E1F74093660142E04093680171D00D
:104460004F914395403671F7089540E0E0E0F0E960
:104470004F934093660142E040936801709364015A
:104480005DD0CCE3DFE00E947A7932964F9143957C
:10449000403671F7789408950E9424014F9340911B
:1044A000340140936D014CE440933401C6E0DAE0FE
:1044B000E7E1FCE00E9432350E94A2330B075772FD
:1044C0006974696E6720646174612E2E2E004091BC
:1044D0006D01409334014F910C941D01C6E3C6E376
:1044E00040914501942F4F5C499340E249934BE53D
:1044F0004993409131014F934068409331010E94AC
:10450000AC794DE549934F914093310108950E9454
:10451000623F08950E942A400E94003E08950E9432
:10452000A93D08950E942E3E08950E94413F08959E
:104530000E94BF3F08950E94324008950E94A84003
:1045400008950E944E4008950E94B73D08950E942C
:10455000DB3E0895A1E00E94AB3720923201209209
:104560004601A7E00E940931C0E0D0E0EDE1F6E1AC
:104570000E946A35A0E70E9409310E94A23301021D
:104580004156522D436869704261736963322063FA
:104590006F6E6669677061676500A7E00E94093108
:1045A0000E94A2331401436865636B73756D3A20F2
:1045B000000021D159D0E8E5F8E4E8940E94F237F0
:1045C000413009F413C1423059F44091140151E0D3
:1045D0004527409314010E9407790E94F623EACFF1
:1045E000433059F44091140152E04527409314019F
:1045F0000E9407790E94F623DDCF443059F44091A0
:10460000140154E04527409314010E9407790E9449
:10461000F623D0CF453059F44091140158E0452796
:10462000409314010E9407790E94F623C3CF4730BC
:1046300049F40E941A79439547700E9415790E94A7
:10464000F623B8CF483059F44091140150E1452782
:10465000409314010E9407790E94F623ABCF4A30A1
:1046600011F40E94492D76CFA6E00E9409310E94E4
:10467000A23303014B6579626F617264206C6179CA
:104680006F75743A00000E94A23305015365726988
:10469000616C2073706565643A000E94A233070163
:1046A0004932432073706565643A00000E94A2336A
:1046B00009015350492073706565643A00000E94F7
:1046C000A2330B01454550524F4D20616464726521
:1046D00073733A000E94A2330D014C696E65204548
:1046E0006E643A00A1E70E9409317091140170FDD7
:1046F0000AC00E94A2330312444520285157455254
:10470000545A290009C00E94A2330312555320288D
:10471000515745525459290071FD0AC00E94A233D5
:10472000051220313230302042707320200009C041
:104730000E94A233051220323430302042707320A0
:10474000200072FD0AC00E94A233071220203130DF
:1047500030206B487A20200009C00E94A233071243
:104760002020343030206B487A20200073FD0AC0AE
:104770000E94A23309122020202035204D487A20A3
:10478000200009C00E94A2330912202031353620B2
:104790006B487A2020000E94A2330B122020202098
:1047A00020000E941A794770405D0E9410320E94DA
:1047B000A233FF2020202020000074FD0AC00E94A8
:1047C000A2330D1220202043522B4C4620202000E3
:1047D00009C00E94A2330D1220204C46206F6E6C3F
:1047E00079202000A7E00E9409310895A0911E01C0
:1047F000A030E1F70895AA27BB27CC27DD27EE27B5
:10480000FF27159042E0149EA00DB11DC21DD21DC0
:10481000459147E0149EA00DB11DC21DD21DFE386A
:1048200081F7EE27F0EF459141E7149EB01DC11DC1
:10483000D21D459147E0149EB01DC11DD21DF03020
:1048400091F7BF93AF93DE019FE00E948C31AF914F
:10485000BF910E948C310895204578697420204BC7
:104860006579622020536572202020493243202040
:104870002053504920202020202020204545505200
:104880004F4D204C696E6520202020202020436C55
:104890006F6E6520AEE0A0933401C1E0D4E0ECE19E
:1048A000F2E10E9432350E94A233050500000E9409
:1048B0007C020E94A23306032020202020286329A6
:1048C00020323030362D3230303920202020202048
:1048D00000000E94A2330703202020206279204A92
:1048E0006F65726720576F6C6672616D20202020A3
:1048F0000000A2EAA09334010E94A2330903202001
:104900002020202044656469636174656420746FAD
:1049100020202020202000000E94A2330A03466CA1
:104920006F7269616E2C204572696B20616E642024
:104930004469616E612E0000AEE0A09334010E94D4
:10494000A2330C025468697320736F6674776172C6
:1049500065206973206C6963656E736564000E94ED
:10496000A2330D04756E64657220746865207465E9
:10497000726D73206F662074686520000E94A233F8
:104980000E04474E55205055424C4943204C494354
:10499000454E534520562E3220000E94A2330F036D
:1049A00055736520697420617420796F7572206F6A
:1049B000776E207269736B210000A2ECA093340122
:1049C0000E94A233110720505245535320414E59A3
:1049D000204B455920000E942E36089561E00E9428
:1049E000DB3750911E015D3E09F408954531B1F762
:1049F00090914501E0E0F0E99770929540EC949F2A
:104A0000E00DF11DCCE3DDE050E0459149935A956E
:104A1000E1F7CCE3DDE00E94D03C0E94DB3750910F
:104A20001E015D3E11F34630A1F76395CCEBDDE04E
:104A30000E94D03C0E94DB3750911E015D3EA9F2DE
:104A40004630A1F763956931E9F644E00E94BF372B
:104A50000895909145019770E0E0F0E9929540EC5F
:104A6000949FE00DF11D45E10E94BF3760E06F9318
:104A7000CCE3DFE00E94AD3C803041F0813051F169
:104A8000883241F145E10E94BF37F2CF46E00E94F3
:104A9000BF37CCEBDFE00E94AD3C803041F081308D
:104AA000C9F08832B9F045E10E94BF37F2CF0E94C9
:104AB0007A797894329646E00E94BF376F91639579
:104AC0006C30A9F60E94CB374430E1F746E00E94F3
:104AD000BF3708956F91089561E00E94DB375091D0
:104AE0001E015D3E09F408954531B1F7A0E8762F27
:104AF0007A95A79FE001ACE3BDE070E80E94633DBA
:104B00004D937A95D9F7CCE3DDE00E94D03C0E942A
:104B1000DB3750911E015D3E31F34630A1F76395BE
:104B20006F3021F744E00E94BF37089545E10E94AD
:104B3000BF3760E06F93CCE3DDE00E94AD3C803096
:104B400031F0883201F145E10E94BF37F4CFA0E88F
:104B5000762F7A95A79FE001ACE3BDE070E84D9118
:104B60000E946C3D7A95D9F746E00E94BF376F915D
:104B700063956E30F9F60E94CB374430E1F746E09A
:104B80000E94BF3708956F91089502414253282E25
:104B90002E2E0353474E282E2E2E04535152282ECC
:104BA0002E2E054E4F54282E2E2E06524E44282EC1
:104BB0002E2E07414443282E2E2E08494E282E2EF5
:104BC0002E2E09585045454B282E0A54454D502845
:104BD0002E2E0B4C4F282E2E2E2E0C4849282E2ED2
:104BE0002E2E0D4B4559282E2E2E0E455045454B49
:104BF000282E0F455252282E2E2E104152282E2E8E
:104C00002E2E1153494E282E2E2E12434F53282E4E
:104C10002E2E134654595045282E144653495A45B2
:104C2000282E155053544154282E16535049282EDF
:104C30002E2E174D454E55282E2E185642595445A6
:104C4000282E1958524543282E2E805052494E5432
:104C50002E2E81434C532E2E2E2E82474F544F2EF4
:104C60002E2E83424F582E2E2E2E8441434F5059C4
:104C70002E2E8553594E432E2E2E86454E442E2ED3
:104C80002E2E8742434F50592E2E885448454E2E83
:104C90002E2E89504F532E2E2E2E8A4E4F54452E97
:104CA0002E2E8B4F4E53594E432E8C52524541441B
:104CB0002E2E8D5257524954452E8E474F535542F2
:104CC0002E2E8F52455455524E2E90564D4F4445E0
:104CD0002E2E914E4558542E2E2E92494E505554FC
:104CE0002E2E93504C4F542E2E2E94574149542E15
:104CF0002E2E95545345542E2E2E96544745542E01
:104D00002E2E974653454C454354984F4E4552528C
:104D10002E2E99535055542E2E2E9A534745542ECD
:104D20002E2E9B45504F4B452E2E9C4745545049A7
:104D3000582E9D434952434C452E9E434F4C4F5253
:104D40002E2E9F424F524445522EA0464F4E542E77
:104D50002E2EA150554D502E2E2EA258504F4B4561
:104D60002E2EA356504F4B452E2EA44C494D495440
:104D70002E2EA547455443484152A644524157540C
:104D80004F2EA7504C41592E2E2EA8535052495405
:104D9000452EA95343524F4C4C2EAA425245414BEB
:104DA0002E2EAB464153542E2E2EAC534C4F572E25
:104DB0002E2EAD445241572E2E2EAE49434F4D4D0F
:104DC0002E2EAF444154412E2E2EB04354455854FC
:104DD0002E2EB146524541442E2EB24657524954CA
:104DE000452EB343424F582E2E2EB44745544154BE
:104DF0005452B54644454C455445B646424F582E4C
:104E00002E2EB750414C45545445B8464F522E2E85
:104E10002E2EB949462E2E2E2E2EBA4449522E2E13
:104E20002E2EBB4F55542E2E2E2EBC464349524398
:104E30004C45BD414C4552542E2EBE464352454131
:104E40005445BF41534B2E2E2E2EC03F2E2E2E2EBC
:104E50002E2EC15853454E442E2EC742432E2E2E81
:104E60002E2ECA4E4F2E2E2E2E2ECC5252442E2E89
:104E70002E2ECD5257522E2E2E2ECE474F532E2E43
:104E80002E2ECF5245542E2E2E2EC2474F2E2E2E72
:104E90002E2ED0564D2E2E2E2E2ED2494E502E2E48
:104EA0002E2ED3504C2E2E2E2E2ED74653454C2E22
:104EB0002E2EDC4750582E2E2E2EDD43492E2E2E20
:104EC0002E2EDE434F4C2E2E2E2EDF424F2E2E2E18
:104ED0002E2EE258502E2E2E2E2EE356502E2E2EF3
:104EE0002E2EE44C494D2E2E2E2EE54743482E2ED5
:104EF0002E2EE644544F2E2E2E2EE85350522E2E98
:104F00002E2EED44522E2E2E2E2EEE49432E2E2ED8
:104F10002E2EEF44412E2E2E2E2EF14652442E2EB2
:104F20002E2EF24657522E2E2E2EF44741542E2E60
:104F30002E2EF54644454C2E2E2EF750414C2E2E4B
:104F40002E2EFC4643492E2E2E2EFE4643522E2E4A
:104F50002E2E002E2E2E2E2E2E2EA0911001B09130
:104F60001101ED01E2EBF2E0CE0FDF1FF6EFE09171
:104F70001601FE0F7F934F92EEE14E2E6991ED9157
:104F80005491762F7295762757FD672768B9ED9172
:104F9000000056FD76B9049055FD76B96991162E3C
:104FA00054FD76B91294162653FD76B907FC612597
:104FB0004A9452FD76B9502D712D41F76091170139
:104FC00068B94F907F91EE91F0911601F395FA3008
:104FD00029F4FF27A0931001B0931101F09316015B
:104FE0000C949B2FA0911001B0911101D091000160
:104FF000C0910101C295DC0FDE7EE5E11090170142
:10500000FD914D2FF0FD429548B900004D2FF1FD67
:10501000429548B900004D2FF2FD429548B9000075
:105020004D2FF3FD4295000048B96D2F4D2FF4FD33
:10503000429548B9CD91F5FD62955D2F68B9F6FDB1
:1050400052956D2F4D2F58B9F7FD6295C0FD4295D1
:10505000000068B9FC2FEA95B9F618B8EE91F09106
:105060001601F395F23029F4FF27A0931001B093B5
:105070001101F09316010C949B2FA0911001B09197
:105080001101D1E0FEE110901701ED91CE2FC37018
:10509000588158B9CE2FC695C695C3705881E295F0
:1050A00058B9CE2FC3705881CE2FC69558B9C69522
:1050B000C3705881ED91CE2F58B9C3705881FA95BD
:1050C00041F718B8EE91F0911601F395F33029F4F9
:1050D000FF27A0931001B0931101F09316010C94D7
:1050E0009B2FA0911001B09111010F931090170107
:1050F000EAE2D1E0CD91C6950C2FC295C770F88138
:10510000F8B9C02F0000C770F8810000000000004F
:10511000F8B9CD91C6950C2FC295C770F881EA9564
:1051200079F718B811970F91F0911601F395F430B3
:1051300029F4FF27A0931001B0931101F0931601F9
:105140000C949B2FA0911001B0911101D0910001FE
:10515000C0910101C295DC0FDE7EE0E110901701E5
:10516000FD914D2FF0FD429548B900000000000070
:105170004D2FF1FD429548B90000000000004D2F71
:10518000F2FD429548B9000000004D2FF3FD429515
:10519000000048B9000000006D2F4D2FF4FD42952E
:1051A00048B90000CD91F5FD62955D2F68B900000A
:1051B0000000F6FD52956D2F4D2F58B9F7FD629501
:1051C000C0FD42950000000068B9FC2F00000000FF
:1051D000EA9551F6000018B8EE91F0911601F3959A
:1051E000F33029F4FF27A0931001B0931101F0933D
:1051F00016010C949B2FA0911001B0911101C09148
:105200004901D82DF6EFE0911601FE0FE395E093EA
:105210001601EA3088F1EC3069F59396A0931001FD
:10522000B093110120921601DC3031F4D091480185
:10523000D09349010C949B2FD83189F4ADE3B2E0AF
:10524000C0913601D3E2CD9FA00DB11DCFE0A09358
:105250001001B0931101C09349010C949B2FD83DCC
:1052600049F4CBE4AAE1B2E0A0931001B09311019C
:10527000C09349010C949B2F0F931F932F93D83DFC
:1052800028F4DC2F0C2F1C2F2C2F05C029E61DE243
:1052900008E8DCECCBE46C2F7C2F7295ED91E7FDF8
:1052A0006727EF775491ED9168B9172E56FD16B820
:1052B0006C2F7C2F729555FD16B8E7FD672754FDBE
:1052C00016B8EF77000053FD16B8049052FD16B8DB
:1052D000502DED9168B9172E56FD16B86C2F7C2F06
:1052E000729555FD16B8E7FD672754FD16B8EF77A0
:1052F000000053FD16B8049052FD16B8502DED91E4
:1053000068B9172E56FD16B86C2F7C2F729555FD77
:1053100016B8E7FD672754FD16B8EF77000053FD78
:1053200016B8049052FD16B8502DED9168B9172E9D
:1053300056FD16B86C2F7C2F729555FD16B8E7FDFB
:10534000672754FD16B8EF77000053FD16B8049098
:1053500052FD16B8502DED9168B9172E56FD16B8AE
:105360006C2F7C2F729555FD16B8E7FD672754FD0D
:1053700016B8EF77000053FD16B8049052FD16B82A
:10538000502DED9168B9172E56FD16B86C2F7C2F55
:10539000729555FD16B8E7FD672754FD16B8EF77EF
:1053A000000053FD16B8049052FD16B8502DED9133
:1053B00068B9172E56FD16B86D2F7D2F729555FDC5
:1053C00016B8E7FD672754FD16B8EF77000053FDC8
:1053D00016B8049052FD16B8502DED9168B9172EED
:1053E00056FD16B86D2F7D2F729555FD16B8E7FD49
:1053F000672754FD16B8EF77000053FD16B80490E8
:1054000052FD16B8502DED9168B9172E56FD16B8FD
:105410006D2F7D2F729555FD16B8E7FD672754FD5A
:1054200016B8EF77000053FD16B8049052FD16B879
:10543000502DED9168B9172E56FD16B86D2F7D2FA2
:10544000729555FD16B8E7FD672754FD16B8EF773E
:10545000000053FD16B8049052FD16B8502DED9182
:1054600068B9172E56FD16B86D2F7D2F729555FD14
:1054700016B8E7FD672754FD16B8EF77000053FD17
:1054800016B8049052FD16B8502DED9168B9172E3C
:1054900056FD16B86D2F7D2F729555FD16B8E7FD98
:1054A000672754FD16B8EF77000053FD16B8049037
:1054B00052FD16B8502DED9168B9172E56FD16B84D
:1054C0006D2F7D2F729555FD16B8E7FD672754FDAA
:1054D00016B8EF77000053FD16B8049052FD16B8C9
:1054E000502DED9168B9172E56FD16B8602F702F0C
:1054F000729555FD16B8E7FD672754FD16B8EF778E
:10550000000053FD16B8049052FD16B8502DED91D1
:1055100068B9172E56FD16B8602F702F729555FD7D
:1055200016B8E7FD672754FD16B8EF77000053FD66
:1055300016B8049052FD16B8502DED9168B9172E8B
:1055400056FD16B8602F702F729555FD16B8E7FD01
:10555000672754FD16B8EF77000053FD16B8049086
:1055600052FD16B8502DED9168B9172E56FD16B89C
:10557000602F702F729555FD16B8E7FD672754FD13
:1055800016B8EF77000053FD16B8049052FD16B818
:10559000502DED9168B9172E56FD16B8602F702F5B
:1055A000729555FD16B8E7FD672754FD16B8EF77DD
:1055B000000053FD16B8049052FD16B8502DED9121
:1055C00068B9172E56FD16B8602F702F729555FDCD
:1055D00016B8E7FD672754FD16B8EF77000053FDB6
:1055E00016B8049052FD16B8502DED9168B9172EDB
:1055F00056FD16B8612F712F729555FD16B8E7FD4F
:10560000672754FD16B8EF77000053FD16B80490D5
:1056100052FD16B8502DED9168B9172E56FD16B8EB
:10562000612F712F729555FD16B8E7FD672754FD60
:1056300016B8EF77000053FD16B8049052FD16B867
:10564000502DED9168B9172E56FD16B8612F712FA8
:10565000729555FD16B8E7FD672754FD16B8EF772C
:10566000000053FD16B8049052FD16B8502DED9170
:1056700068B9172E56FD16B8612F712F729555FD1A
:1056800016B8E7FD672754FD16B8EF77000053FD05
:1056900016B8049052FD16B8502DED9168B9172E2A
:1056A00056FD16B8612F712F729555FD16B8E7FD9E
:1056B000672754FD16B8EF77000053FD16B8049025
:1056C00052FD16B8502DED9168B9172E56FD16B83B
:1056D000612F712F729555FD16B8E7FD672754FDB0
:1056E00016B8EF77000053FD16B8049052FD16B8B7
:1056F000502DED9168B9172E56FD16B8612F712FF8
:10570000729555FD16B8E7FD672754FD16B8EF777B
:10571000000053FD16B8049052FD16B8502DED91BF
:1057200068B9172E56FD16B8612F712F729555FD69
:1057300016B8E7FD672754FD16B8EF77000053FD54
:1057400016B8049052FD16B8502DED9168B9172E79
:1057500056FD16B8622F722F729555FD16B8E7FDEB
:10576000672754FD16B8EF77000053FD16B8049074
:1057700052FD16B8502DED9168B9172E56FD16B88A
:10578000622F722F729555FD16B8E7FD672754FDFD
:1057900016B8EF77000053FD16B8049052FD16B806
:1057A000502DED9168B9172E56FD16B8622F722F45
:1057B000729555FD16B8E7FD672754FD16B8EF77CB
:1057C000000053FD16B8049052FD16B8502DED910F
:1057D00068B9172E56FD16B8622F722F729555FDB7
:1057E00016B8E7FD672754FD16B8EF77000053FDA4
:1057F00016B8049052FD16B8502DED9168B9172EC9
:1058000056FD16B8622F722F729555FD16B8E7FD3A
:10581000672754FD16B8EF77000053FD16B80490C3
:1058200052FD16B8502DED9168B9172E56FD16B8D9
:10583000622F722F729555FD16B8E7FD672754FD4C
:1058400016B8EF77000053FD16B8049052FD16B855
:10585000502DED9168B9172E56FD16B8622F722F94
:10586000729555FD16B8E7FD672754FD16B8EF771A
:10587000000053FD16B8049052FD16B8502DED915E
:1058800068B9172E56FD16B8622F722F729555FD06
:1058900016B8E7FD672754FD16B8EF77000053FDF3
:1058A00016B8049052FD16B8502DED9128B82F91DE
:1058B0001F910F910C949B2FA0911001B091110199
:1058C000E6E8F4E0C0911601D3E0CD9FE00DF11DB4
:1058D0007F936EE17EE1C7E1D1E05881507F452F93
:1058E0004295542B588358B952954D914F7358B9DE
:1058F0005991469F58B95295EF01000058B9C00D13
:10590000D11D599158B952957A950000000058B9A7
:10591000599149F7000058B952956091170100005C
:1059200058B959917F9158B95295F0911601F39554
:1059300058B90000000068B9FA3029F4FF27A09395
:105940001001B0931101F09316010C949B2FA4ED5C
:10595000B1E0C0E1D2E0809216010C94B627A2EF2C
:10596000B1E0CEE2D2E0425D409316010C94B6273E
:10597000482D4A5008F4EBCF423D08F0F0CF58E1F3
:105980004695ACE4B2E0A40FB21D4C91459FA5EB47
:10599000B2E0A00DB11DCEE655274D91C39556B985
:1059A000D9F1C417D9F75D9158B9C3954D91529566
:1059B000C39556B989F1C417D9F75D9158B9C39504
:1059C0004D915295C39556B939F1C417D9F75D91E8
:1059D00058B9C3954D915295C39556B9E9F0C4177E
:1059E000D9F75D9158B9C3954D915295C39556B964
:1059F00099F0C417D9F75D9158B9C3954D91529557
:105A0000C39556B949F0C417D9F75D9158B9C395F4
:105A10004D915295C39556B9B1F1C417D9F75D911F
:105A200058B9C3954D915295C39556B961F1C417B4
:105A3000D9F75D9158B9C3954D915295C39556B913
:105A400011F1C417D9F75D9158B9C3954D9152958D
:105A5000C39556B9C1F0C417D9F75D9158B9C3952C
:105A60004D915295C39556B971F0C417D9F75D9110
:105A700058B9C3954D915295C39556B921F0C417A5
:105A8000D9F75D9158B9509117010000000058B93D
:105A900052C20E94DD3A6F436C6F6E65207379735A
:105AA00074656D3F2000413009F0089565D087D0BE
:105AB000803079F078D00E94B43A4F4E6F20636FF7
:105AC0006E74726F6C6C657220666F756E64200008
:105AD00008958DD0803069F066D00E94B43A4F4E60
:105AE0006F204D65676136343420666F756E6400D3
:105AF0000895CDD09DD0EE27FF2750E060E00590BF
:105B0000B8D00590BDD063956038C9F79ED0539545
:105B1000A9F74CEA4ED040EA4CD04AD046EE49D0E4
:105B20000E9405360E9405360E9405364CEA41D097
:105B300048EA3FD03DD041ED3CD00E9405360E945E
:105B400005360E9405364CEA34D044EA32D030D0D3
:105B50004CEF2FD00E9405360E9405360E94053674
:105B600022D00E94B43A8053797374656D20636CBF
:105B70006F6E65640000089543E54CBD2DBC249A0A
:105B80002C984FEF4A95F1F72C9A4FEF4A95F1F781
:105B90002C984FEF4A95F1F72C984FEF4A95F1F773
:105BA0000E94053608952C9A4CE54CBD3DBC0895E5
:105BB00044274EBD4DB547FFFDCF4EB5089588270C
:105BC0004CEAF7DF43E5F5DFF3DF433509F081E029
:105BD000EFDF0895BF93AF934F93A42FBB270E948D
:105BE0008C310E940F324F91AF91BF910895882759
:105BF00040E3DFDFDDDF40E0DCDFDADF4E3111F0F4
:105C000082E0089540E3D5DFD3DF41E0D2DFD0DF8B
:105C1000463911F082E0089540E3CBDFC9DF42E06E
:105C2000C8DFC6DF493019F04A3009F082E0089534
:105C30004CEABFDF40E8BDDFBBDFBADF0E940536BC
:105C40000E9405360E94053608954CE4B2DF452FC8
:105C50004695AFDF452F440F440F440F440F440FC8
:105C6000440F440FA6DFA4DF0E9405360E940536CC
:105C7000089540E49EDF9CDF462F9BDF402D99CFA7
:105C800048E497DF95DF462F94DF402D92CF0E94A6
:105C900024014F934091340140936D014CE44093B3
:105CA0003401C5E0DAE0E8E1FCE00E9432350E9410
:105CB000A2330B06436C6F6E696E67205379737461
:105CC000656D2E2E2E0040916D01409334014F9151
:105CD0000C941D0128B818954F935F936F93FF9311
:105CE000EF93DF93CF93BF93AF930F921F92FFB7C2
:105CF000FF9330921901B0913901B7FF5C98B7FD5D
:105D00005C9A4B99BE7F4B9BB160B0933901C0E167
:105D1000D1E05F89A889E9890A881B88A00DE11D67
:105D2000A88BE98BFFA14491AD89AF73AF3309F420
:105D3000452F5AA54503B0E8B10DB093B300EE89E5
:105D4000FF89488D598DAA27E2FDA095E5FDA09514
:105D5000F4FDA09557FDA095AA1FEE1FFF1F441F3D
:105D6000551FEE8BFF8B488F598F830C921CEBA92C
:105D7000FF81EF23E8B97894E9A190FC04C0F8A56D
:105D80008F1608F4A9C071F4409108014F3F51F0FB
:105D900040910A014A9521F44091090130920B018A
:105DA00040930A01FCE0E2FFFDEE8F1639F45E98A5
:105DB000E3FFC1C0B2E8B0938000BDC0F1E1E2FFF3
:105DC000F3EF8F1639F45E9AE3FFB5C0B2ECB093EF
:105DD0008000B1C0FBE1E2FFFFEF8F1621F4EFEF8F
:105DE000E0934301A8C0F2E0E2FFF9EE8F1619F448
:105DF00020924301A0C0F9E3E2FFF7E08F1609F01B
:105E00009AC0A4EDA883A1E0A9832E8288249924B6
:105E1000AAE0A9AFA5E0E2FFA39542E3E2FF4CE3CD
:105E2000BA8DB395BA1731F4BB27EB8DFC8D319643
:105E3000EB8FFC8FBA8FE885E395E41709F4EE2722
:105E4000E887FDE8E0E0A0912501A7FDB096AC89C8
:105E5000EA0FF21DB491B21511F0A395AC8BBAA75D
:105E6000A0915801A03009F466C0B0915901B395D2
:105E7000B0935901BA17C0F320925901B091600153
:105E8000BA95B093600181F7E0915A01F0915B01FE
:105E9000C0915E01D0915F012196A191B191B09323
:105EA0006001E0935A01F0935B01B8D6FD1798F0BA
:105EB000EC1788F0A0913B01A13029F4A2E02092D8
:105EC0005801A0933B01E0915C01F0915D01E093EA
:105ED0005A01F0935B012FC0A0918400A63EE0F32D
:105EE000A73E00F0A83E00F0A93E00F0AA3E00F058
:105EF000E5FD21C0E0913101E7FD0C94FB28E09124
:105F00004601E53011F40C94A228E03011F40C9411
:105F1000AD27E13011F40C94F227E23011F40C9427
:105F20003D28E43011F40C945C2CE63011F40C9410
:105F3000B82C0C947128A0911C01A5FD27C0E091FC
:105F4000C000E7FF6BC0E091C600E0937D01F5EF74
:105F5000B491B0FF36C0A7FF03C020921E015BC002
:105F6000E33809F4E0E1F6E84091140140FDFE5FFA
:105F7000EF77A4FFA6FDF395A4FFA0FDE068A1FDC7
:105F8000E068E491E0931D01A06246C0E0911D012C
:105F9000E0931E01E0931F01EE3E19F4A2FD0C9464
:105FA000EF0040913501E33611F4A2FD4160E03786
:105FB00011F4A3FD4260EC3F09F4446040933501C5
:105FC0002AC0E03F11F4A06827C0E03E11F4A064AD
:105FD00023C0E23131F4A6FD1EC0A160A7FDAE7F53
:105FE0001AC0E93521F4A260A7FDAD7F14C0E431E9
:105FF00051F4A6FD04C0A460A7FDAB7F0CC0A8604F
:10600000A7FDA77F08C0E13121F4A061A7FDAF7E05
:1060100002C020921E01AF71A0931C014091140197
:1060200041FD0E94A17841FF0E94D678FF91FFBFF9
:106030001F900F90AF91BF91CF91DF91EF91FF91A2
:106040006F915F914F911895AAEBA4B9AFEFA5B9E5
:10605000A0EEA7B9A0E0A8B9A0EFAAB9AFEFABB97D
:10606000A6B1AF77A0933101B2ECB0938000B9E153
:10607000B0938100F4E0A2FFF4E0F0938700FEEF1C
:10608000A2FFF6EFF093860020928900FAE5F093E4
:106090008800F4E0F0938B00F8EDF0938A00A6E01E
:1060A000A0936F00A2E0A4BDA1E0A5BDA1E3A7BDA0
:1060B000A3E8A093B000A1E0A093B100A0E8A09352
:1060C000B3002092B6002092C000A0E1A093C100CE
:1060D000A6E6A093C200ACE5B0911401B3FDAFE514
:1060E000ACBDA0E0ADBDA5E194D0C0E1D1E0A4ED90
:1060F000A993A1E0A993AEE12992AA95E9F7AAEAAA
:10610000A0932601A093280120923201209215012C
:10611000AEE3A09324010F93009131010F77009318
:10612000310106EE07C00F93009131010068009322
:10613000310104EE009338010F910895A0934601B8
:10614000A03041F4ACE3A0934C01AEE2A0934D012A
:10615000A6EE44C0A13069F4A8EAA0934C01A4E7DC
:10616000A0934D01A0E0A0930001A0EEA093010137
:1061700024C0A23091F4A8E7A0934C01ACE4A09312
:106180004D01C0E0D1E0A0E0A993A0E4A993A0EA6A
:10619000A993A0EEA993A3EE21C0A33081F4A4E5B6
:1061A000A0934C01AAE3A0934D01C0E0D1E0AA273F
:1061B000B8E0A993A05EBA95E1F7A7EE0FC0A530AD
:1061C00081F4A0E8A0934C01A0E4A0934D01A0E2CB
:1061D000A0930001A0EEA0930101A0ECA0933801D0
:1061E0000895A43051F4ACE3A0934C01AEE2A09327
:1061F0004D010E948C38A6EEF1CFACE3A0934C0188
:10620000A2E0A0934D010E94C8380E94D438A6EEA7
:10621000E5CFAA0FAE7EA09334010895A295AA0FF0
:10622000A07EA0931701089548834091310147FD56
:1062300017C040914601443099F0CF93DF935F93AC
:106240005CE3C50FD21D463021F046E7C40F42E0A3
:10625000D41F409134014E7E48835F91DF91CF91EE
:1062600008954F935F936F93AF93BF9340E2592F7D
:106270005370523061F0533009F44BE2B7FF05C060
:10628000A095B095A30DB21D4DE20E941032592F7A
:106290005C70692F6073E8944FE24395A051B74258
:1062A000E0F7A05FB84D5C3009F42BD04FE2439586
:1062B000A85EB340E0F7A851BC4F53FD22D0603335
:1062C00009F4ABD04FE24395A456B209E0F7AC59BC
:1062D000BF4F503009F015D0603209F49ED04FE224
:1062E0004395AA50E8F70DD0A65F603109F495D028
:1062F00040E34A0F95D0BF91AF916F915F914F915D
:106300000895403311F068948BC091FD89C0F6F375
:1063100090FF089584C008954F9390FF05C04B2FC0
:10632000429509D04B2F07D04A2F429504D04A2FCF
:1063300002D04F9108954F70405D4A3308F0495F95
:106340006FC0409146014030C9F0AF93BF93CF93E7
:10635000DF93D1E0C4EDA7E1443009F0ACE5BEE144
:106360002992BA95E9F7AA95D1F7DF91CF91AA249E
:10637000BB2420923301BF91AF910895AF93BF9397
:10638000CF93DF9340E2D1E0C4EDA7E1BEE14993B2
:10639000BA95E9F7AA95D1F7409134014E7EA7E16D
:1063A000BEE14993BA95E9F7AA95D1F7DF91CF916C
:1063B000AA24BB2420923301BF91AF910895AF93DB
:1063C000BF9320923301A0913201A03051F4A7E194
:1063D000AA24B394AB1571F7B6E1BB2ECF93DF932C
:1063E0006AC0A13021F4BF91AF910C94B337A230B1
:1063F00049F44DE0B0911401B4FFB8D4BF91AF910E
:106400004AE0B4C4A33019F4BF91AF910895BF918D
:10641000AF915AE00E94F33C08954CE201C040E283
:10642000AF93BF93A0913301A395A0933301A091A3
:106430003201A43030F0BF91AF91542F0E94F33C51
:106440000895A030A9F0A33059F4A42FBB275F937F
:106450006F930E94CD186F915F91BF91AF91089596
:10646000BF91AF91A0913201A1FF0C94BF377EC4C0
:10647000EF93E0914601E03029F0E63019F0E43086
:1064800009F09AC0EF91CF93DF9354D496FD35C0B5
:10649000CBDEA395AE3131F4AA27B395B73111F411
:1064A000B6E107C0AA2EBB2EDF91CF91BF91AF916D
:1064B0000895AA2EBB2ED1E0C4ED4F93A6E1BEE114
:1064C0004E8D4993BA95E1F7AA95C9F7AEE140E23E
:1064D0004993AA95E9F7D4E0C6E8A6E1BEE14E8D5E
:1064E0004993BA95E1F7AA95C9F7AEE14091340115
:1064F0004993AA95E9F74F91D7CFAB31A8F6B231BE
:1065000098F6AD5FAA2EEF93FF934F925F926F9232
:106510007F9270F85F93E42FF6EFB5E044245524A2
:1065200066245527A491A7FD539550FB40F8A6FD7E
:10653000539550FB41F8A5FD539550FB50F8A4FD31
:10654000539550FB51F8A3FD539550FB60F8A2FD05
:10655000539550FB61F8F3955527A491A7FD5395EA
:1065600050FB42F8A6FD539550FB43F8A5FD53950B
:1065700050FB52F8A4FD539550FB53F8A3FD5395DF
:1065800050FB62F8A2FD539550FB63F8F395442D40
:106590004BDE2196452D48DE2196462D45DE6C9634
:1065A000BA9509F0BBCF5F9170FA7F906F905F90C2
:1065B0004F90FF91EF9178CFFF93CF93DF936F933D
:1065C0007F93E42F6091150160FD1EC0F6EFAA2DA8
:1065D000BB2DDAE0C49137D0B395AA2D96FD33D008
:1065E00096FDB395F395AA2DDA95A1F7AA2DAA5F8A
:1065F00096FDAA5FAA2E7F916F91DF91CF91FF91B7
:10660000EF91BF91AF910895F1E8EF77AE2FECEFE6
:10661000EA0FF21DAA0FEA0FF21DAA2DBB2DD6E03C
:10662000C49155D0B395AA2D96FD51D096FDB39542
:10663000D0FD3196AA2DDA9599F7AA2DAC5F96FD7B
:10664000AC5FAA2ED8CF609134016F936295C7FDDD
:10665000629560933401A2D0A39596FD9FD096FDDC
:10666000A395C6FD62956093340198D0A39596FDDD
:1066700095D096FDA395C5FD6295609334018ED0AB
:10668000A39596FD8BD096FDA395C4FD629560936E
:10669000340184D0A39596FD81D096FDA395C3FDCA
:1066A0006295609334017AD0A39596FD77D096FDDC
:1066B000A395C2FD62956093340170D0A39596FDB9
:1066C0006DD096FDA3956F9160933401089560910C
:1066D0003401D0FDC295762FC7FF729570933401B7
:1066E0005DD0A39596FD5AD096FDA395762FC6FF53
:1066F00072957093340152D0A39596FD4FD096FDBC
:10670000A395762FC5FF72957093340147D0A3955A
:1067100096FD44D096FDA395762FC4FF7295709395
:1067200034013CD0A39596FD39D096FDA395609396
:10673000340108954F934591403011F44F910895DD
:106740006FDEF9CFFF91EF91EE0FFF1FAF93BF9375
:10675000B591BF3F11F0A5910ED0BF91AF914F936E
:106760004591403031F44F913197F695E795319648
:10677000099456DEF5CFEF93E0914601E03021F029
:10678000EF91AA2EBB2E0895EF91AE3108F0ADE146
:10679000B73108F0B6E1AA2EBB2E0895CF93DF9350
:1067A000C0914C01CA1728F0C0914D01CB1708F0D9
:1067B00003C0DF91CF910895AF93BF934F935F9341
:1067C000C0914601C53031F0C43041F0C37039F09A
:1067D000C23008F442C009F465C082C099C051E0DB
:1067E000AC3360F5BE3250F5B0FD550FB0FD550F1E
:1067F000A0FD550FB695A695CEE1BC9FD1E0C4EDA6
:10680000CA0FD21DC00DD11DA2EBB2E0CA0FDB1F13
:10681000A881B0913401BE70B295A07EBA17A9F0DC
:10682000B0913401BE70AB2BAE7EA883A2EBB2E078
:10683000CA1BDB0BB881B52BBF70B8835F914F913A
:10684000BF91AF91DF91CF910895A2EBB2E0CA1B47
:10685000DB0BB8815095B523EFCFCA2FC770C39516
:1068600040E00894441FCA95E9F7A695A695A69519
:10687000C5E1D0914601D2FDC0E1BC9FD1E0C4ED9D
:10688000CA0FD21DC00DD11DA0913401A695A170D3
:1068900029F44095A881A423A883D0CFA881A42B54
:1068A000A883CCCFCA2F509134015695537043E042
:1068B000C37031F0440F440F550F550FCA95C9F7F7
:1068C0004095A695A695CEE1BC9FD1E0C4EDCA0F38
:1068D000D21DC00DD11DA881A423A52BA883AECFA6
:1068E000CA2F509134015E704EE0C17011F4429590
:1068F00052954095A695CAE2BC9FD1E0C4EDCA0F5F
:10690000D21DC00DD11DA881A423A52BA88396CF8D
:1069100051E0AC33D0F4BE32C0F4B0FD550FB0FD41
:10692000550FA0FD550FB695A695CEE1BC9FD1E0C1
:10693000C4EDCA0FD21DC00DD11DB0913401B2708B
:1069400029F0B881B52BBF70B88378CFB881509546
:10695000B523F9CFCE3108F0CDE1EE3108F0EDE10D
:10696000D73108F0D6E1F73108F0F6E1EC1718F46A
:106970000E2EEC2FC02DFD1718F40F2EFD2FD02D4D
:106980000895EC1718F40E2EEC2FC02DFD1718F4F7
:106990000F2EFD2FD02D0895AF93BF93CF93DF938C
:1069A000EF93FF935F93D6DFAC2FBD2FCF93DF9391
:1069B000C3D1288252EBC50F52E0D51F509134014C
:1069C0005883DF91CF91AE1711F0A395EFCFBF178A
:1069D00019F0AC2FB395EACF5F91FF91EF91DF9162
:1069E000CF91BF91AF910895AF93BF93CF93DF93B2
:1069F000EF93FF935F93C5DFAC2FBD2FCFDEA39541
:106A0000AE17E1F7CBDEB395FB17E1F7C7DEAA952A
:106A1000AC17E1F7C3DEBA95BD17E1F75F91FF91BF
:106A2000EF91DF91CF91BF91AF910895AF93BF9355
:106A3000CF93DF93EF93FF935F93A3DFBD2FAC2F33
:106A4000ADDEAE1711F0A395FBCFA8DEFB1711F05A
:106A5000B395F5CF5F91FF91EF91DF91CF91BF910A
:106A6000AF91089599DFAF93BF93CF93DF93EF93E7
:106A7000FF934F935F936EDF4C2FBD2FAC2F5CD1F4
:106A800052EF599351EFA395AE1711F05993FBCFE5
:106A900053EF5993A42FB395BF1739F04DD150EF51
:106AA0005993AE2F49D15993F5CFA42F45D154EF27
:106AB000599351EFA395AE1711F05993FBCF55EFB2
:106AC00059935F914F91FF91EF91DF91CF91BF91DA
:106AD000AF910895C7DF5F93AF93BF93CF93DF93D9
:106AE000EF93FF9337DFBD2FAC2F26D15BEF599388
:106AF0005CEEA395AE1711F05993FBCF5CEF599361
:106B0000FF91EF91DF91CF91CF93DF93EF93FF93BD
:106B1000BD2FAC2FB39510D15DEF599350E2A395E3
:106B2000AE1711F05993FBCF5EEF5993FF91EF91A0
:106B3000DF91CF91CF93DF93EF93FF93BD2FAC2FD6
:106B4000B395AF93F9D0A2EBB2E0CA0FDB1F50911F
:106B5000340152955E7E2196AF91A395AE1711F048
:106B60005993FBCFFF91EF91DF91CF91CF93DF93BB
:106B7000EF93FF93BD2FAC2FBE5FDED05EEE599337
:106B80005DEEA395AE1711F05993FBCF5FEE5993CD
:106B9000FF91EF91DF91CF91BF91AF915F910895F8
:106BA0000F931F932F933F93AF93BF93CF93DF9395
:106BB000DE010FEFCE1B10F40195C1951FEFDF1B17
:106BC00010F41195D195CD1760F000C02C2F2695AB
:106BD000E5DDAE1789F0A00F2D1BD0F7B10F2C0FFC
:106BE000F7CF2D2F2695DADDBF1731F0B10F2C1B13
:106BF000D0F7A00F2D0FF7CFDF91CF91BF91AF91BD
:106C00003F912F911F910F910895AF93A82DA73E0B
:106C1000E9F3A82DA73EE9F7AF910895EF93FF930D
:106C2000AF93A0932501FBE8A6FDFCE8F0933701A4
:106C3000AF73AA0FFDE8E0E8EA0FF21DA591A0935B
:106C40002201A591A09323012092240120922001EA
:106C500020922101AF91FF91EF91089520921F01A1
:106C600040911F014030E1F3BCC040911E01403013
:106C7000E1F708955FD0A2EBCA0FA2E0DA1FA88166
:106C8000BA2FAF93A171BE7EB295BA2BAF9120926D
:106C90001F0140911F01403041F4409118014B31D8
:106CA00010F4A883F6CFB883F4CFA8839AD042C05B
:106CB0003F933DED52D020921F0140911C01447042
:106CC000431749F0403021F40E94CC07342F03C011
:106CD0000E94F207342F40911F01403061F440912F
:106CE00018014B3120F448814F774883E6CF488123
:106CF00040684883E2CF58815F7758833F91089579
:106D0000D1E0CFEDCA0FD21D20921F0140911F018B
:106D1000403061F4409118014B3120F448814F77A5
:106D20004883F4CF488140684883F0CF58815F772B
:106D300058830895AA2DBB2DDEE1BD9FD1E0C4ED9F
:106D4000CA0FD21DC00DD11D0895F6DF0F9302EBBF
:106D5000C00F02E0D01F0F910895D3E2BD9FD2E093
:106D6000C0E4CA0FD21DC00DD11D0895BF93BFEF5F
:106D7000B1B900001A99FECF42B9B4E6BA95F1F75D
:106D80002998B4E6BA95F1F7299ABF91089546E596
:106D9000F6D00E94B337C4EDD1E0F4E0EEE1D2D0FA
:106DA000FA95E9F7F3E0E3E2CDD0FA95E9F7F9E6F1
:106DB000E8E1C8D0FA95E9F70BC045E5E0D00E94BC
:106DC000B337C4EDD1E0F7E5EEE1BCD0FA95E1F7D9
:106DD000CF91DF91EF91FF914F91442708954F910B
:106DE00008954F934091350141FFF9CF4D7F409376
:106DF000350140914601463090F7FF93EF93DF93C2
:106E0000CF934430D1F2403029F44091310147FF13
:106E100013C025C04F9347E4B2D04F914F93405DCC
:106E2000AED04F91413009F447C0423009F453C00D
:106E3000433009F465C06DC044E50E94BF370E942D
:106E4000B337C4EDD1E0FEE2EEE17CD0FA95E1F794
:106E5000CF91DF91EF91FF914F914427089545E441
:106E60000E94BF374091480163D00E94B337C4ED00
:106E7000D1E0F3E0E3E266D00E94B337FA95D1F7B0
:106E8000E3E2F0913601EF9FC00DD11DF0E1E3E2A6
:106E900048814F7742954FD049914F774CD0EA9532
:106EA000B9F70E94B337FA9591F7CF91DF91EF913F
:106EB000FF914F91442708954091000139D04091AE
:106EC000010136D050D0C4EDD1E0F4E7E5E13AD08D
:106ED000FA95E1F7EACF409100012AD040910101F3
:106EE00027D04091020124D04091030121D03BD012
:106EF000C4EDD1E0F4E5EEE125D0FA95E1F7D5CF88
:106F000032D0C4EDD1E0FAE3EAE21CD0FA95E1F721
:106F1000CCCF409100010CD04091010109D023D089
:106F2000C4EDD1E0F0E4E0E10DD0FA95E1F7BDCF9A
:106F30004295469547704F70405D4A3308F0495F6F
:106F40000C94BF3748814295F6DF4991F4DFEA950A
:106F5000C9F70C94B337BF93B2E0A03009F0B06426
:106F6000B4BDBF910895BF934F934DE0B09114010C
:106F7000B4FF05D04AE003D04F91BF910895BF936D
:106F8000B0912D01B030E1F740932E01BA95B09346
:106F90002D01BF910895BF93B0912F01B030E1F75B
:106FA000BA95B0932F01B0912F01B030E1F7409125
:106FB0003001BF910895BF93B0912F01B030E1F738
:106FC000BA95B0932F0140911E014D3E41F0B09112
:106FD0002F01B030C1F740913001BF9108954BE1CE
:106FE000BF910895DF93CF93BF93AF93FF93EF9338
:106FF000CAE1D7E0ECE6F0E733D0EF91FF91FF93E1
:10700000EF93EFDEC8E6D4E0B0911C01B2FD7E96AE
:1070100016F026D001C01ED040911E01A1E04D3EC9
:1070200069F0A2E0413F51F0A3E0423F39F0A4E013
:10703000433F21F0A5E0443F09F0DFCFB0911C01B0
:10704000B2FDAB5F4A2FEF91FF91AF91BF91CF910E
:10705000DF910895BEE1A191A993BA95E1F7089552
:10706000BEE1A591A993BA95E1F708954E4E4E4E13
:107070004E4EC0C0C0C0C0C08080808080802E2E98
:107080002E2E2E2E6E6E6E6E6E6EDF93CF93BF938E
:10709000AF93FF93EF93CAE1D7E0ECE6F0E7E0DFD0
:1070A000EF91FF91FF93EF93C8E6D4E0D9DFCBCF08
:1070B000ACE5B0911401B3FDAFE5ACBDACE5A09378
:1070C000B800A0E0B2FDA1E0A093B9000895FF933D
:1070D000EF930F93E0912601A0912701B091280131
:1070E000F09129010027E2FD0095E5FD0095A4FD42
:1070F0000095F7FD0095001FEE1FAA1FBB1FFF1F85
:10710000E0932601A0932701B0932801F093290171
:107110000F91EF91FF910895DF93CF93BF93AF93BA
:10712000FF93EF934F935F936F937F93A4EDB1E041
:10713000C2EBD2E02D922197E9F740E050E0E0E089
:10714000F6EFF50FE40F6491C0913401DC2FD29576
:10715000C07FD07FE3E0772711D072950FD0729572
:107160007D93EA95C1F753955A3049F743954034DA
:1071700029F77F916F915F914F9165CF67FF05C0B0
:107180004F934C2FCD2FD42F4F917C2B660F08950A
:10719000DF93CF93BF93AF93CCE4D2E0A1E4BAE006
:1071A00029921197E9F751CFDF93CF93BF93AF9314
:1071B000C4EDD1E0ACE3B0E2009034010CAEB99381
:1071C000AA95E1F742CF0E9424014F935F936F93FA
:1071D0007F934F925F926F927F922F9320914601FF
:1071E00040904E01509051016090500170905301B9
:1071F00050914F0160915201A22FA370E52F660FAD
:10720000EE0FA33031F0660FEE0FA23011F0660FD3
:10721000EE0FF62FA0915401A13071F4E20142D09B
:10722000803011F08FE133C0E3013CD0803011F0A9
:1072300080E22DC060D02BC0A23091F4E20132D0A8
:10724000803011F08FE123C0E3013BD0803011F09A
:1072500082E11DC0ACE3BDE06A0E7B1E70D017C09A
:10726000A33011F085E113C0A52DA33010F082E109
:107270000EC0ACE3BDE04A0E5B1EF201519161917C
:10728000E30110D0803011F080E201C062D02F9174
:107290007F906F905F904F907F916F915F914F9132
:1072A0000C941D01CE0F10F48FE10895A0914C01B4
:1072B000CA17D0F7DF0FC0F3B0914D01DB17A0F76D
:1072C0000895659FC00DD11D2296D33008F082E14C
:1072D0000895A22F50914F0160915201E52F660F42
:1072E000EE0FA33031F0660FEE0FA23011F0660FF3
:1072F000EE0FF62F0895571478F0D20134D0ECE851
:10730000FBE064D0D3012FD0ECE8FBE084D05394B1
:1073100073946A9591F70895560E760E5A947A945E
:10732000D20121D0ECE8FBE051D0D3011CD0ECE835
:10733000FBE071D05A947A946A9591F70895F3011D
:1073400051936193D2010FD041D053946A95D1F7F4
:107350000895F20151916191D30105D05CD07394ED
:107360006A95D1F708956F93C4EDD1E0213011F4FF
:1073700065E103C0253069F460E1B69FC00DD11D01
:107380006A2F669566956695C60FD21D4A2F6F9136
:107390000895223069F46EE1B69FC00DD11D6A2FA9
:1073A00066956695C60FD21D4A2F440F6F910895BA
:1073B0006AE2B69FC00DD11D6A2F66956695C60F0D
:1073C000D21D4A2F440F440F6F9108957F936F93FE
:1073D000BF93AF93652F742F777029F4A991A19370
:1073E0006A95E1F73FC0B0E8713019F0B6957A952B
:1073F000FBCF7727A991AB9F703019F0A291A029FC
:10740000A193119273957617A9F7A991AB9FA291B9
:10741000A029A19327C07F936F93BF93AF93652F4C
:10742000742F777029F4A191A9936A95E1F71AC096
:107430000F931F930FEF11E0000F110F7A95E1F7F3
:10744000652F7881009570230095A191A19F072A4F
:107450000992712D6A95C9F768816023672B69933A
:107460000F911F91AF91BF916F917F9108950E94ED
:1074700024010F931F932F9310E020E0FAE8EE27EA
:10748000C0914F01CF77D0915201DF7704910C9FCB
:10749000A12DE0950491E0950D9FB12DA11729F440
:1074A000B21719F4E39591F724C01A2F2B2FA0914E
:1074B0004E01B0915101A10FB20F0E94CE33A091A5
:1074C0004E01B0915101A10FB21B0E94CE33A09189
:1074D0004E01B0915101A11BB21B0E94CE33A0916D
:1074E0004E01B0915101A11BB20F0E94CE33E39522
:1074F00069F62F911F910F910C941D010E94240198
:107500000F931F932F933F932FEFFAE8EE27C0912D
:107510004F01CF77D0915201DF7704910C9FA12DBD
:10752000E0950491E0950D9FB12DB21721F4E395FC
:10753000A1F73F91DECF1A2F2B2FA0914E01B091D2
:1075400051013A2FB21BA11B310F0E94CE33B20F53
:10755000B20F0E94CE33B21BB21BA3953A17A8F705
:10756000E395D9F63F91C5CFFF91EF91EE0FFF1F45
:107570005BD03197F695E7953196EF93FF93C4E88A
:10758000D1E0409134014F93FF93EF9361D00E947B
:10759000A2330B0920505245535320454E544552B7
:1075A0002000EF91FF914F914093340157DB4A3E09
:1075B000E9F75BDB0E94C71B0895FF91EF91EE0F87
:1075C000FF1F32D03197F695E7953196EF93FF93F1
:1075D000C4E8D1E0409134014F93FF93EF9338D04A
:1075E0000E94A2330B08202859296573202F2028D8
:1075F0004E296F200000EF91FF914F91409334018D
:107600002DDB493761F0493551F04E3619F04E34D3
:1076100009F0F6CF2ADB0E94C71B4427089525DB1B
:107620000E94C71B41E00895C4E8D1E0459146950A
:107630004F93477049934F9142954770499358E152
:1076400045914993403011F05A95D1F72992089508
:10765000FF93EF9392E020923201A991B991B295F4
:10766000B077A770AB0FAA0FA0933401DF93CF932D
:107670000E94A51BC2E0D8E0EBE1FCE00E9432359D
:10768000A3E0B9E00E94BB33CF91DF9158E149916B
:10769000403051F0DF93CF935F930E9410325F919F
:1076A000CF91DF915A9599F74091340142954093DB
:1076B0003401EF91FF9108950E942401C0914E0181
:1076C000D09151010A8119810E3118F4173108F453
:1076D00015D0A0915001B0915301C0914E01D091AD
:1076E0005101B983AA83AE3138F4B73128F438D0C8
:1076F0007370713009F071D00C941D01C0914E016E
:10770000D09151010A8119812C813B81239F310F36
:107710002596C00DD11DC00DD11D412FE4EDF1E026
:107720005EE1549FE00DF11DE00FF21D522F6991B3
:1077300061935A95E1F74395431781F7412FE6E8A6
:10774000F4E05EE1549FE00DF11DE00FF21D522FB9
:10775000699161935A95E1F74395431781F708952D
:10776000C0914E01D09151010A8119812C813B8138
:10777000239F310F2596C00DD11DC00DD11D772738
:10778000412FE4EDF1E05EE1549FE00DF11DE00FCB
:10779000F21D522F619169936F7009F071E05A9553
:1077A000C9F74395431769F7E0914E01F0915101F4
:1077B0004081742B7083412FE6E8F4E05EE1549F32
:1077C000E00DF11DE00FF21D522F619169935A9562
:1077D000E1F74395431781F70895C0914E01D09189
:1077E00051010A8119812C813B81310F2596412F4E
:1077F000E4EDF1E05EE1549FE00DF11DE00FF21DBC
:10780000522F699161935A95E1F74395431781F798
:10781000412FE6E8F4E05EE1549FE00DF11DE00F3A
:10782000F21D522F6991660F28F46E70462E60810A
:10783000607F642961935A95A9F74395431749F7E7
:1078400008950E9424014F935F936F93E091340158
:10785000437001F5A2E1B2E0C0E3D2E0F22D0BD01B
:10786000A0914601A43031F0A4ECB4E0C2EED4E023
:10787000FE2F01D06DC062E15AE149914D935A95B6
:10788000E1F7149624966A95B9F75AE1FD935A9553
:10789000E9F708954130E9F4A8E4B4E0C7E4D4E09E
:1078A000F22D0BD0A0914601A43031F0AAEFB6E042
:1078B000C9EFD6E0FE2F01D04BC063E159E14A91F8
:1078C0004E935A95E1F7FE93149725976A95B1F771
:1078D0000895423001F5A8E4B4E0CAE2D4E0F22D04
:1078E0000BD0A0914601A43031F0AAEFB6E0CCED68
:1078F000D6E0FE2F01D02CC062E15AE14A914E93AE
:107900005A95E1F7149724976A95B9F75AE1FE93CF
:107910005A95E9F70895A2E1B2E0C3E1D2E0F22D71
:107920000BD0A0914601A43031F0A4ECB4E0C5EC3A
:10793000D4E0FE2F01D00CC063E159E149914D9391
:107940005A95E1F7FD93259614966A95B1F7089537
:107950006F915F914F910C941D014F935F937F93B3
:107960002ADB4B3111F481E015C04130C9F713DB3C
:10797000642F11DB4095641711F088E20BC070E8AA
:10798000552709DB540F49937A95D9F704DB45173E
:1079900029F488277F915F914F91089589E2FACF6A
:1079A0004F935F937F9341E0EADA462FE8DA409500
:1079B000E6DA70E855274991540FE1DA7A95D9F75C
:1079C000452FDDDA7F915F914F9108955E984CE5E8
:1079D0004093B80044E84093BC0044E94093BC00A5
:1079E000089544EA0EC05093BB0044E80AC044EC3A
:1079F00008D05091BB00089544E803D05091BB00DB
:107A000008954093BC004091BC0047FFFCCF6091BB
:107A1000B900687F0895E5DF683089F4572F550F66
:107A20005E70506AE0DF683151F45B2FDCDF683252
:107A300031F45A2FD8DF683211F4882708958FE087
:107A40005F915F91CACFE7DFCCDF603169F4572FD8
:107A5000550F5E70516AC7DF603431F4CDDF683591
:107A600019F411968827B9CF8FE0B7CF052ED3DF51
:107A7000502DB9DF683219F411968827AECF8FE008
:107A80000895AFDF6830A9F4572F5770550F51692B
:107A9000AADF603471F4ABDF603559F4A52FACDF99
:107AA000683539F4BB27550FAA1F08F4B09588270D
:107AB00094CF8FE092CF8827D83020F082E24F9188
:107AC0004F914FEF0895F7DFF999FECFD2BDC1BDB9
:107AD000F89A40B521960895EEDF8827F999FDCFF1
:107AE000D2BDC1BDF89A40B4441611F42196089550
:107AF00040BDF894FA9AF99A7894F999FECFF89AD9
:107B000021960895AF93DFDF4193AA95E1F7AF91F6
:107B10000895AF934191E0DFAA95E1F7AF91089501
:107B20004EBD4DB547FFFDCF4EB5089588272C9823
:107B300047EDF6DF4427F4DF2C9A4C7B4432B1F357
:107B40004C31A1F38827443A19F04C3909F081E10E
:107B500008958827EBDF803021F040E040939C10AF
:107B600008954C3911F448E0F9CF40E1F7CFF1DF47
:107B7000403009F40895440F440F440F440F4A95D0
:107B80000895AA0FBB1F4B2FCBDF4A2FC9DF422D11
:107B9000C7DFB695A7950895803059F44F93C6DF97
:107BA000803031F42C9845E5BBDFEBDF2C9ABEDF4B
:107BB0004F910895803059F44F93B8DF803031F4FD
:107BC0002C9843E5ADDFDDDF2C9AB0DF4F910895AF
:107BD000803051F44F93AADF803029F42C9846E886
:107BE0009FDFCFDF2C9A4F9108951196B0939D108F
:107BF000A0939E101197ECCF2DD2CEDF48D0E8CFC6
:107C00007F93772710D07F9108957F9371E00BD0F9
:107C1000D42F72E008D0C42F7F9108957F9373E032
:107C200002D07F910895803099F480DF803081F414
:107C30002C9842ED75DFAA0FBB1FA3954B2F70DF69
:107C40004A2F6EDF472F6CDFB695A79502D02C9A8E
:107C5000089566DF65DF64DF63DF62CF8030B1F4F3
:107C600065DF803099F42C9842ED5ADFAA0FBB1FD4
:107C70004B2F56DF4A2F54DF472F440F51DFB69565
:107C8000A795E7DFD42F4CDFC42F2C9A08957F935C
:107C900070E010D07F9108957F9371E04D2F0AD04E
:107CA00072E04C2FC0DF7F9108957F9373E0BBDFBC
:107CB0007F9108958030A1F44F9338DF4F91803049
:107CC00079F42C984F9347E82BDF442729DF41E0D4
:107CD00027DF472F25DF4F914F9322DF2C9A4F91BB
:107CE0000895803091F422DF8030D1F72C984F93A3
:107CF00047E816DF442714DF40E012DF472F10DF8C
:107D00004F914F930DDF2C9A4F9108958030D1F40D
:107D1000DF93CF934F935F9309DF803079F42C98F2
:107D200047E8FEDE4427FCDE4427FADE40E0F8DECA
:107D300055274991F5DE5A95E1F72C9A5F914F91BD
:107D4000CF91DF9108958030B1F44F935F93EEDED1
:107D5000803079F42C9847E8E3DE4427E1DE4427BD
:107D6000DFDE40E0DDDE55274FEFDADE5A95E1F742
:107D70002C9A5F914F9108958030E1F4DF93CF9377
:107D80004F935F93D3DE803089F42C9846EDC8DEA4
:107D90004427C6DE4427C4DE40E0C2DE4427C0DEFE
:107DA0005527BEDE49935A95E1F72C9A5F914F9182
:107DB000CF91DF910895BF93AF93DF93CF934F930C
:107DC0005F937F93C6DE403001F4BDDF4FE05FDF9D
:107DD00044276BDFAA27BB27FBDE11964DEFCA2F86
:107DE000CF70C13009F44CEF52DF44275EDFCC275F
:107DF000DD2752DFEDDE1196A03019F445EE0E942A
:107E0000103240919C10B41749F70AC0BF93AF934A
:107E1000DF93CF934F935F937F939BDE403091F43A
:107E20007F915F914F91CF91DF91AF91BF91089575
:107E3000B42FAA271197F2DEC42FBB27AA27EEDEA4
:107E40004C1731F4A9DEEADE43952FDFC1DEE8CF1F
:107E50001196E4DE4C17E1F7F5CFDF93CF934F9304
:107E60009BDE4DEFCA2FCF70C13009F44CEF0FDF0E
:107E7000CCDE219611DF67DFABDE4F91CF91DF9132
:107E80000895FF93EF93DF93CF93BF93AF93AA2708
:107E9000BB27ED015EDE4030A1F0F42FB1DE4C3F98
:107EA00041F04D3F31F04B3A21F04F3018F040395E
:107EB00008F421961196BF1789F74427DF1709F4B4
:107EC00041E06FC00F93BF93AF934F93AA27BB2797
:107ED000ED01FD013EDE403099F0042F91DE4D3F73
:107EE00049F4DF93CF9391DE4D2FCF91DF914F3F38
:107EF00021F021964C3F09F431961196B01771F795
:107F00004F91AF91BF910F910895FF93EF93DF933E
:107F1000CF934F932F931DDE4030A9F0AA27BB27A4
:107F20006FDE242FB0919D10A0919E104091100102
:107F3000B41710F0A2E0BB27FD0162DE4D3F31F423
:107F400064DED21718F42F914F912DC015964091F1
:107F50009C10B41709F4BB27BF1779F7AE1769F760
:107F6000AA27BB2719DE4CDE4F3F31F0405F242F9C
:107F70008EDE2EDEDF01E1CFAFEFBFEFE4CFFF9368
:107F8000EF93DF93CF93BF93AF934F935F936F9331
:107F90007F93DFDD403061F481E17F916F915F91EC
:107FA0004F91AF91BF91CF91DF91EF91FF910895E4
:107FB00051D0B41710F08BE1F0CF22DE4C3F11F01E
:107FC00087E1EBCF40916601403011F48BE1E5CFC2
:107FD000413810F08BE1E1CF75DFD03021F4C417C8
:107FE00010F488E1DACFCCE8DBE050E06FEF699382
:107FF0005A95E9F7A8DE1196B0939D10A0939E10B4
:1080000040916601CCE8DBE04F937FDFB993A99301
:108010004BEA3DDEDF93CF93F8DD21963DDECF9135
:10802000DF91FCDD42DEE1DDF1DE4F914A9561F743
:1080300011D0CCE8DBE06ADE4091680128DEDF93F6
:10804000CF93E3DD219628DECF91DF91E7DD2DDEB2
:10805000BFDDA3CFA0916401A295BA2FA07FBF700E
:10806000119608950E9424014F935F937F93772781
:10807000F1DFC6DD4C3F69F0F1DDDF3F49F0BF9332
:10808000AF93DE01EADEAF91BF91C0DE7F5FA1F763
:10809000E4DE7F915F914F910C941D010E942401B9
:1080A0004F935F937F932F93AA27BB273FDDA8DDD4
:1080B000242FD0DFA5DD4C3F39F489E12F917F914A
:1080C0005F914F910C941D0170916601703810F012
:1080D0008BE1F4CFC3DDDF3F11F48BE1EFCFDE01A5
:1080E000CCE3DDE040916801413009F4D3954230A2
:1080F00009F4DE5F0BDEDF93CF9387DDD21759F0F3
:108100002196CADDCF91DF917BDDC1DD87DDCDDD3D
:108110005FDD7CDED3CFA1DEF8DE77DD2196BCDD2E
:10812000CF91DF914BEAB3DD79DDBFDD51DDED01AC
:1081300091DF32DD70916601770F4D2FD2DD73959F
:108140004C2FCFDD5DDDA3DD69DDAFDD41DDB6CFD9
:108150000E9424014F935F937F937CDF51DD4C3F5E
:1081600031F48EE17F915F914F910C941D017091DC
:108170006601703810F08BE1F5CF70DDDF3F11F450
:108180008BE1F0CFDE0108DDCCE3DDE0409168015A
:10819000413009F4D395423009F4DE5FEDDDE2CFE2
:1081A0000004080D11161A1F23282C3035393D42C2
:1081B000464A4F53575B5F64686C7074787C7F836A
:1081C000878B8F92969A9DA1A4A7ABAEB1B5B8BB91
:1081D000BEC1C4C6C9CCCFD1D4D6D9DBDDDFE2E481
:1081E000E6E8E9EBEDEEF0F2F3F4F6F7F8F9FAFB76
:1081F000FCFCFDFEFEFFFFFFFFFFFFFF000000CCC9
:10820000C000333000FFF000000CCCCCCCCC333CB1
:10821000CCFFFCCC000333CCC333333333FFF33315
:10822000000FFFCCCFFF333FFFFFFFFFA5A5A50643
:10823000FF600000000000000000000000000000DF
:10824000000000000000000000000000000000002E
:108250000EAE000004E000AAE800EE4E000000446C
:108260004040AA000066FF666842C4A248A0000021
:10827000004400004888404222400A4A0004E400CA
:1082800000048000E000000040224880EAAAE04CA0
:1082900044E0E2E8E0E2E2E0AAE220E8E2E0E8EA44
:1082A000E0E24880EAEAE0EAE2E004040004048054
:1082B0002484200E0E00842480C268E400EEE04A8C
:1082C000AEA0CACAC0688860CAAAC0E8C8E0E8C848
:1082D0008068EA60AAEAA0E444E0E22A60AC8CA0EC
:1082E0008888E0AEAAA0CAAAA04AAA40EAE8804AC2
:1082F000AA60EAECA068E2C0E44440AAAAE0AAAA04
:1083000040AAAEA0AA4AA0AA4440E248E064446061
:1083100004A400C444C04A00000000E04400004A35
:10832000AEA0CACAC0688860CAAAC0E8C8E0E8C8E7
:108330008068EA60AAEAA0E444E0E22A60AC8CA08B
:108340008888E0AEAAA0CAAAA04AAA40EAE8804A61
:10835000AA60EAECA068E2C0E44440AAAAE0AAAAA3
:1083600040AAAEA0AA4AA0AA4440E248E024C42001
:0C8370004444448464808842208CEC80EB
:1086000000F900F5F3F1F2FC00FAF8F6F4EB5E0085
:10861000F7000000007131000000797361773200CB
:108620000063786465343300002076667472350028
:10863000006E6268677A360000006D6A7537380030
:10864000002C6B696F303900002E2D6C00707E009D
:1086500000000000002700000000EA2B00230000BB
:10866000003C00000000EC00003100343700000046
:10867000302C32353638ED00FB2B332D2A390000F3
:1086800000F900F5F3F1F2FC00FAF8F6F4EB000063
:10869000F70000000051210000005953415722000B
:1086A00000435844452440000020564654522500BB
:1086B000004E4248475A260000004D4A552F2800D8
:1086C000003B4B494F3D2900003A5F4C00503F00B2
:1086D00000000000006000000000EA2A00270000FF
:1086E000003E00000000EC000031003437000000C4
:1086F00030E932353638ED00FB2B332D2A390000B6
:108700000000000000000000000000000000000069
:108710000000000000000000000000000000000059
:108720000000000000000000000000000000000049
:1087300000000000000000C000000000000000C1B8
:10874000000000000000000000002F0000000000FA
:1087500000000000000000000000EA000000C2006D
:10876000000000000000000000E100E2E000000066
:10877000E8E9E500E3E4ED00FB2BE72D2AE6000045
:1087800000000000000000000000000000000000E9
:108790000000000000400000000000000000000099
:1087A00000000000000000000000000000000000C9
:1087B000000000000000000000000000007B5B00E3
:1087C00000000000007D5D000000000000007E0051
:1087D00000000000000000000000005C000000003D
:1087E000007C00000000000000E100E2E00000006A
:1087F000EFEEE500E3E4ED00FB2BE72D2AE60000B9
:1088000000F900F5F3F1F2FC00FAF8F6F4EB5E0083
:10881000F70000000071310000007A7361773200C8
:108820000063786465343300002076667472350026
:10883000006E62686779360000006D6A753738002F
:10884000002C6B696F303900002E2F6C3B702D00AF
:10885000000027005B3D00000000EA5D007E000094
:10886000000000000000EC00003100343700000080
:10887000302C32353638ED00FB2B332D2A390000F1
:1088800000F900F5F3F1F2FC00FAF8F6F4EB000061
:10889000F70000000051210000005A5341574000EA
:1088A00000435844452423000020564654522500D6
:1088B000004E424847595E0000004D4A55262A00A6
:1088C000003C4B494F292800003E3F4C3A505F0086
:1088D000000022007B2B00000000EA7D007C0000ED
:1088E000000000000000EC00003100343700000000
:1088F00030E932353638ED00FB2B332D2A390000B4
:108900000000000000000000000000000000000067
:108910000000000000000000000000000000000057
:108920000000000000000000000000000000000047
:1089300000000000000000C000000000000000C1B6
:10894000000000000000000000002F0000000000F8
:1089500000000000000000000000EA000000C2006B
:10896000000000000000000000E100E2E000000064
:10897000E8E9E500E3E4ED00FB2BE72D2AE6000043
:1089800000000000000000000000000000000000E7
:1089900000000000000000000000000000000000D7
:1089A00000000000000000000000000000000000C7
:1089B00000000000000000000000000000000000B7
:1089C00000000000000000000000000000000000A7
:1089D0000000000000000000000000000000000097
:1089E000000000000000000000E100E2E0000000E4
:1089F000EFEEE500E3E4ED00FB2BE72D2AE60000B7
:108A0000FFFFFFFFFFFFFFFFFFFFFFFEFEFEFEFE7B
:108A1000FEFEFDFDFDFDFDFCFCFCFCFBFBFBFBFA93
:108A2000FAFAF9F9F9F8F8F8F7F7F6F6F6F5F5F4D1
:108A3000F4F3F3F2F2F2F1F0F0EFEFEEEEEDEDEC35
:108A4000EBEBEAEAE9E8E8E7E6E6E5E4E4E3E2E1BD
:108A5000E1E0DFDEDEDDDCDBDADAD9D8D7D6D5D46B
:108A6000D4D3D2D1D0CFCECDCCCBCAC9C9C8C7C63A
:108A7000C5C4C3C2C1BFBEBDBCBBBAB9B8B7B6B529
:108A8000B4B2B1B0AFAEADACAAA9A8A7A6A5A3A237
:108A9000A1A09E9D9C9B99989796949392918F8E5E
:108AA0008D8B8A898786858382817F7E7D7B7A789C
:108AB0007776747371706F6D6C6A696766656362EF
:108AC000605F5D5C5A595756545351504E4D4B4A56
:108AD0004847454442413F3E3C3B393836353332C6
:108AE000302E2D2B2A2827252422201F1D1C1A1941
:108AF00017161412110F0E0C0B09070604030100C0
:108B00000C11161A1E2225282B2D2F313233333407
:108B100034343434343434343535363738393B3CF6
:108B20003E40434547494B4D4F5152535454545482
:108B3000545351504E4C4A4745423F3D3A383634E3
:108B40003231302F2E2E2E2F303132333536383A07
:108B50003C3E4042444647494A4B4D4E4E4F505092
:108B60005050505050504F4E4D4C4B494846434149
:108B70003E3B37332F2B27221D18130D0802FDF81B
:108B8000F3EEE9E5E1DDDAD7D4D2D0CECDCCCCCB53
:108B9000CBCBCBCBCBCBCBCBCACAC9C8C7C6C4C344
:108BA000C1BFBCBAB8B6B4B2B0AEADACABABABAB98
:108BB000ABACAEAFB1B3B5B8BABDC0C2C5C7C9CB17
:108BC000CDCECFD0D1D1D1D0CFCECDCCCAC9C7C5D3
:108BD000C3C1BFBDBBB9B8B6B5B4B2B1B1B0AFAF28
:108BE000AFAFAFAFAFAFB0B1B2B3B4B6B7B9BCBE51
:108BF000C1C4C8CCD0D4D8DDE2E7ECF2F7FD02075F
:108C0000000A141D272F383F464B505457595959C5
:108C1000585654504C48433E39332E2925201C19B0
:108C200016141211111112131517191C1F222527C2
:108C30002A2C2E303132323232312F2D2B28252260
:108C40001F1C191613110F0D0C0B0A0A0A0B0C0E20
:108C500010121416181A1C1E1F2020201F1E1C196B
:108C600016120D0803FDF7F0EAE3DDD6D1CBC6C23C
:108C7000BFBDBBBABBBCBEC2C6CBD1D7DFE6EFF728
:108C80000008101920282E34393D41434445444200
:108C9000403D39342E29221C150F0802FCF7F2ED55
:108CA000E9E6E3E1E0DFDFDFE0E1E3E5E7E9EBED83
:108CB000EFF1F3F4F5F5F5F4F3F2F0EEECE9E6E3B9
:108CC000E0DDDAD7D4D2D0CECDCDCDCDCECFD1D37D
:108CD000D5D8DADDE0E3E6E8EAECEDEEEEEEEDEB3A
:108CE000E9E6E3DFDAD6D1CCC6C1BCB7B3AFABA9F6
:108CF000A7A6A6A6A8ABAFB4B9C0C7D0D8E2EBF57B
:108D000080675342352B221C16120E0C09070605EC
:108D1000040000000000000000000000000000004F
:108D2000807E7B79777572706E6C6A686664636149
:108D30005F5D5C5A5857555352504F4D4C4B494804
:108D40004745444341403F3E3D3C3B39383736354B
:108D50003433323231302F2E2D2C2B2B2A29282838
:108D60002726252524232322222120201F1F1E1DE4
:108D70001D1C1C1B1B1A1A19191818181717160076
:108D8000890091009A00A300AD00B700C200CE0098
:108D9000DA00E700F4000301120123013401460167
:108DA0005A016E0184019B01B301CD01E901060264
:108DB0002502450268028C02B302DC020803360376
:108DC00067039B03D2030C0449048B04D0041905E8
:108DD0006705B90510066C06CE063507A307170808
:108DE000930815099F09320ACD0A720B200CD80C82
:108DF0009C0D6B0E460F2F1025112A123F13641481
:108E0000F894A0E02A2EA1E03A2EA0E1AEBFAFEF89
:108E1000ADBFB0E0A0E0AA95F1F7BA95D9F7AAEBFB
:108E2000A4B9AFEFA5B9A0E8A7B9A0E0A8B9A0EF91
:108E3000AAB9AFEFABB9A6B1AF71A09331014B990D
:108E40005DC0B2ECB0938000B9E1B0938100F4E072
:108E5000A2FFF4E0F0938700FEEFA2FFF6EFF0939D
:108E6000860020928900FAE5F0938800A2E0A093A2
:108E70006F00A0E4A4BDA1E0A5BDA1E3A7BD209221
:108E8000C000A0E1A093C100A6E6A093C200E0EA62
:108E9000FFE87ED0A2E2B591B993AA95E1F705B7B4
:108EA000036005BF0E7F05BF7894A8EC68D0B09131
:108EB000C600B83719F0AA95C9F720C0E0ECFFE862
:108EC00067D045E140D0C4EDD1E020D046E03BD0B2
:108ED000E0E0F0E0CCE3DFE019D046E034D0CCEBCA
:108EE000DFE014D0FE3820F40E947A79329678942C
:108EF00046E029D0AAEEB1E01BD0ECCFF89405B73C
:108F0000016005BF0C7F05BF0C94000028D04430E1
:108F100039F446E018D0B0912D01B030E1F7EECF32
:108F200050E81DD01CD01BD049935A95E1F717C0CB
:108F30004F2F429501D04F2F4F70405D4A3308F0BC
:108F4000495F4D930895BF93B0912D01B030E1F783
:108F500040932E01BA95B0932D01BF910895BF9310
:108F6000B0912F01B030E1F7BA95B0932F01B091D5
:108F70002F01B030E1F740913001BF910895AF93D8
:108F8000A82DA73EE9F3A82DA73EE9F7AF910895D4
:108F9000C4EDD1E0A2E2B591B993AA95E1F70895A5
:108FA0004156522D436869704261736963322028CB
:108FB0004631313D557064617465205379732920C1
:108FC000426F6F746C6F61646572204572726F726C
:108FD000202845534320746F206578697429202028
:0E900000202020202020202020202020FFFFE4
:0E9C0000202020202020202020202020FFFFD8
:0EA80000202020202020202020202020FFFFCC
:0EB40000202020202020202020202020FFFFC0
:0EC00000202020202020202020202020FFFFB4
:0ECC0000202020202020202020202020FFFFA8
:0ED80000202020202020202020202020FFFF9C
:0EE4000048656C6C6F20576F726C64204EFF85
:10E410000E94A131A0E60E9409310E94A2330000AF
:10E4200048656C6C6F20576F726C64210000A7E028
:10E430000E9409310E94A23302007072657373203A
:0CE4400071000E942E364137E1F708956C
:10F000000C94004700000000000000000000000019
:10F0100000000000000000000000000000000000F0
:10F0200000000000000000000000000000000000E0
:10F03000000000000C941C784F935F936F93FF9334
:10F04000EF93DF93CF93BF93AF930F921F92FFB7CE
:10F05000FF93C0E1D1E0B9A5B7FF5C98B7FD5C9A1A
:10F060004B99BE7F4B9BB160B9A7830C921CE9A161
:10F07000F92DF03029F4F82DFA3010F1F63EF8F0C1
:10F08000FCE0E2FFFDEE8F1639F45E98E3FF17C057
:10F09000B2E8B093800013C0F1E1E2FFF3EF8F1606
:10F0A00039F45E9AE3FF0BC0B2ECB093800007C066
:10F0B000F9E3E2FFF7E08F1611F4882499242CC0BD
:10F0C000A0918400A63EE0F3A73E00F0A83E00F029
:10F0D000A93E00F0AA3E00F0A4EDB1E0F6EFF80D75
:10F0E000C0E2ED91549140E060E848B9ED9156FDE1
:10F0F00066B90000000055FD66B9049054FD66B97C
:10F10000CA95000053FD66B90000000052FD66B9C3
:10F11000502D59F7000028B814D0E091C600E6370A
:10F1200011F40C947E47FF91FFBF1F900F90AF9199
:10F13000BF91CF91DF91EF91FF916F915F914F91CF
:10F140001895A0913901E0912F01E03091F0EF3F47
:10F1500021F4A0FD0EC0EEE30CC0EA95F5EFB491EA
:10F16000B5FF07C0B0913001B695A0FBB7F9B093D9
:10F170003001E0932F01E0912D01E03091F0EF3F5D
:10F1800019F4E0E5AF770DC0EA95F5EFB491B4FF5F
:10F1900008C0B0912E01B0FB0894B795A7F9B093C1
:10F1A0002E01E0932D01A09339010895A09139011A
:10F1B000E0912F01E03091F0EF3F21F4A0FD0EC06F
:10F1C000ECE70CC0EA95F5EFB491B7FF07C0B0913A
:10F1D0003001B695A0FBB7F9B0933001E0932F0151
:10F1E000E0912D01E030E9F2EF3F19F4E0E9AF776B
:10F1F000D8CFEA95F5EFB491B6FFD3CFB0912E01F9
:10F20000B0FB0894B795A7F9B0932E01CACF4091EF
:10F210001401C8EFD7E00E946C3D0895C8EFD7E015
:10F220000E94633D409314010895C9EFD7E00E9406
:10F230006C3D0895CF93DF93C9EFD7E00E94633D03
:10F24000742FDF91CF910895FF93EF93DF93CF93C6
:10F25000AF9301D1E0933C01F0933D01AF91CF9189
:10F26000DF91EF91FF910895E0E0F0E9C0E0DCE08C
:10F27000A42FA03021F0EC0FFD1FAA95FACF08951E
:10F28000E0913C01F0913D01A0E2A99FE00DF11D4C
:10F29000B096CCEAD1E0A0E2B591B993AA95E1F796
:10F2A000BFEFB993089547B740FDFDCFB7BFE895CD
:10F2B00047B740FDFDCF089547B746FF0895B1E138
:10F2C000F2DFFACFF8944E2F407E19F4B3E0EBDF73
:10F2D000F3DFA0E109901990B1E0E5DF3296AA953D
:10F2E000C9F7E03009F008953297B5E0DCDFE4DFDC
:10F2F00032960895F8944F93BF93AF93B3E0D3DF62
:10F30000DBDF3297CCE3DFE0A0E83296099019907A
:10F31000B1E0C9DFAA95C9F7B5E0C5DFCDDFAF9190
:10F32000BF914F910895E0913C01F0913D01B0975C
:10F33000ACE0B591B993AA95E1F7A0913101A7FD91
:10F340000895A6EAB2E0CA0FDB1FACE0B091340129
:10F35000B993AA95E9F70895E0E0F0E9A0E0BCE0F0
:10F36000492F403029F3EA0FFB1F4A95FACF40910D
:10F3700045014770AF93ECE0F0E9ACE0A49FF00DDD
:10F380004491EC50AF910895F89463D0CCEAD1E069
:10F39000AFEDB1E05CE04D9149935A95E1F742E45D
:10F3A000499353E140E2B9935A95E9F7A0978ADF70
:10F3B0009927B3E2B99FA0E4B2E0A00DB11DC4E863
:10F3C000D1E050E24D9149935A95E1F7299250E2EC
:10F3D0004A91403219F428825A95D1F70E94151AA1
:10F3E000CCEAD1E06FDF93959F3519F778940895B3
:10F3F00030D0AFEDB1E05CE045914D935A95E1F727
:10F400007496992750E2ACEAB1E045914D935A9534
:10F41000E1F7A4E8B1E040E253E24D935A95E9F7F1
:10F42000FF93EF939F930E94F71A9F91EF91FF91A3
:10F43000C4E8D1E0B3E2B99FADE3B2E0A00DB11DE5
:10F4400053E249914D935A95E1F793959F35D1F643
:10F45000089540914501AF93BF93E0E0F0E9477014
:10F460004295A0ECA49FE00DF11DBF91AF910895CE
:10F47000CCE3DFE04CE050E259934A95E9F75FEFC7
:10F48000599343E150E259934A95E9F740EF5FEF12
:10F4900059934A95E9F7DDDF2DDF3296CCE3DFE0C3
:10F4A00040E25FEF59934A95E9F74BE04F9322DF33
:10F4B00032964F914A95D1F778940895472F477027
:10F4C000CADFFF93EF93C5DFAF91BF914CE04F933D
:10F4D000CCE3DFE040E0559159934A95E1F7FF9383
:10F4E000EF93FD0107DF3296DF01EF91FF914F911E
:08F4F0004A9569F7789408952C
:10F50000010101010101210101010101012181012B
:10F510000100002100110101010121D101010101BE
:10F520002101110101010121D1010101012101117B
:10F530000101010121D101010101010111010101BB
:10F540000101D1010101010101110101010101C10B
:10F55000010101010101010101000101C1010101DC
:10F56000010101010101010001C1010101010100CD
:10F57000010101010101410001010101010101003D
:10F58000000000400000000000000000000000003B
:10F59000000000000000000000000000000000006B
:10F5A000000000000000000000000000000000005B
:10F5B000000000000000000000000000000000004B
:10F5C000000000000000000000000000000000003B
:10F5D000000000000000000000000000000000002B
:10F5E000100000000000000000000000000000000B
:10F5F00020000000000000000000000000000000EB
:10F60000009010800090108000901080009010807A
:10F61000FC28288004C0145028282800000000007E
:10F6200000000000000000000000000000000000DA
:10F6300000000000000000000000000000000000CA
:10F6400000000000000000000000000000000000BA
:10F6500000000000000000000000000000000000AA
:10F66000000000000000000000000000000000009A
:10F67000000000000000000000000000000000008A
:10F6800028C004C00000000000000000000000804E
:10F69000C0A0888400000000000000002088FCB4A6
:10F6A0000028000008A08080000004C028800024FA
:10F6B00000008000000044288000C004C41800003E
:10F6C000000000000000000000000000C004000076
:10F6D0008090808008A084408080C8A400004C8472
:10F6E000000000000000000080808080008028284A
:10F6F000280000002828002828282800002CE8904E
:10F700000090108000901080009010800090108079
:10F710007C444480A8A814504844440024000000BD
:10F7200000183C3C185028280C3000000000000055
:10F73000241824400C401440242400000C003024E1
:10F7400024244424444040246424106460646424D9
:10F7500044244424406464646464404800481800BD
:10F76000300060000400140060180C6028000000E5
:10F7700000000000300000000000000C18306000A5
:10F7800028A004C0808044283C3C3C000044A88061
:10F79000C0A08884000000000000008040847C58E5
:10F7A000182800001090808004C004C028FC287C29
:10F7B00000440C00000044EC8000C004C42400009D
:10F7C000000000000000000000008080C004000075
:10F7D0008088A41010908440C004C8A400008C80CD
:10F7E000287C008080004084FCF8C004000024488D
:10F7F000280000002828002828282800002CE8C01D
:10F800000090108000901080009010800090108078
:10F81000FC44448080801450444444283C00000050
:10F8200000183C3C20546C181818181800000004EC
:10F830006428640C14603064646428281800186418
:10F84000646464646460606464180C6C605864642C
:10F8500064646464186464646464046000183C0054
:10F860001800600004003400600000601800000010
:10F870000000000030000000000000181818601898
:10F88000449008A0C4C4806C0000001C1844A880E8
:10F89000C0A0888400000000000080804084FCB488
:10F8A0002428282820888080A4A00C60448044401C
:10F8B00000440C40844444800000C0046C24004494
:10F8C00000000000000000000000C004C004481058
:10F8D0008084BCB020888820D834C8A440848C8020
:10F8E0002C7C00C4C4448080C008C00400802088F0
:10F8F000280000002828002828282800002CE8A03C
:10F900000090108000901080009010800090108077
:10F910007C808080808010908480804424186424BF
:10F9200000183C40780C7830300C7C180000000C3B
:10F93000681804183C44600C6464282830400C04A7
:10F94000046464606460606064180C78607C546473
:10F9500064646460186464643C640C60301864001F
:10F960000C2444242C2430207428146C185C742437
:10F970004824742448646464646440181818300C83
:10F9800044881090C4BC446C24246434286C6C807B
:10F99000C0A08884000000000080808080807CEC13
:10F9A000404444442088408490A00C6044FC286477
:10F9B00000440C40844444280000C0046C240080AF
:10F9C00000000000000000000000C004C00418187F
:10F9D0008080BC1040848820E82CC8A480804C849F
:10F9E000EC2400C4EC448080C008C004008020885F
:10F9F000280000002828002828282800002CE8E4F7
:10FA00000090108000901080009010800090108076
:10FA1000FC808080B098109080ECEC44003C6464E2
:10FA20000018003C24183000300C2440004000181E
:10FA30007C180C0C6C044418242000006000040C9A
:10FA40002C6444606444447040180C50607C7C64B6
:10FA50004464442418646464183C18607C180000F2
:10FA6000000464606864486454180C78187C54641A
:10FA70006C6C5460306464643C640C30180C188006
:10FA800080841090C4F8806C04646440406C6C8086
:10FA9000C0A0888400000000808080808080FCB44A
:10FAA0001880442840844084808418308080282432
:10FAB00000440C40844444440000C00428241880BE
:10FAC00000000000000000000000C004C00440244A
:10FAD000A4B0BC4080808080E82CC8A488104084FA
:10FAE000E42400C4EC44D480C008C0048080208892
:10FAF000288020882088808020888020882CE8F03A
:10FB00000000000090909090101010108080808075
:10FB10007C8080801090B098408080440040646475
:10FB2000001800401C307800300C7C182800003091
:10FB300054181804400464186404282830400C1831
:10FB40007C4064606460606464180C78606468641D
:10FB5000607C780418643C7C3C1830600C18000011
:10FB6000002064606440306464180C50187C646445
:10FB70006C6C602430646464182C181818180C0C11
:10FB800080842088C4C444C420646430286C6C80A1
:10FB9000C0A08884000000008080808080807CEC91
:10FBA00018008044408440848080301880FC801895
:10FBB00000448040844444440000C004280024449D
:10FBC00000000000000000000000C004C004244049
:10FBD000BCD0A41084404084E82CC8A44C8480800D
:10FBE000482400C4EC44F880C008C0048080208809
:10FBF000288020882088808020888020882CE82801
:10FC00000000000090909090101010108080808074
:10FC1000FC8080801090808084C4A8440000643CF4
:10FC20000000003C44686C00181818181800286080
:10FC3000641830640C646430640C281818001800D0
:10FC40007C6464646460606464186C6C60646464A4
:10FC500060686C6418643C7C641860600018000084
:10FC6000006464646460302064180C781864646410
:10FC7000482460043C683C7C3C0830181818041880
:10FC800044882088C4C4808064646818186C6C80C0
:10FC9000C0A0888400000080808080808080FCB4C8
:10FCA000400080804084208880843018DC80284098
:10FCB00000446040844444280000C0046C0024C414
:10FCC00000000000000000000000C004C00418187C
:10FCD000BCB0808084402088E44CC4C44C848080C4
:10FCE000282400C4EC44D4D0FCF8C00480002828A8
:10FCF000280028280000280028282820882CE83000
:10FD00000000000090909090101010108080808073
:10FD10007C4480441450808044EC442800004458C3
:10FD20000018003C18082C000C300000300028009F
:10FD3000242440240C242430242800300C003018C3
:10FD4000246444244440602464242864406464247B
:10FD5000602C64241824182464184048004800408B
:10FD6000002044242424300464246C6C246464241F
:10FD7000600C6044182C183C6404400C18300400DB
:10FD8000449040848080442820242C0000A8448093
:10FD9000C0A08884000080808080808040847C585F
:10FDA000240080288080208890A0600CDCFC44180F
:10FDB00000446040844444EC0000C0046C00240013
:10FDC00000000000000000000000C004C004104853
:10FDD000BCB0808080801090D094C0048C8040841F
:10FDE000284000C4C444FCF88080C0048000282857
:10FDF000280028280000280028282820882CE830FF
:10FE00000000000090909090101010108080808072
:10FE1000FC4480441450A8A84080440000006000C6
:10FE200000000000000000000000000000000000D2
:10FE300000000000000000000000000000000000C2
:10FE400000000000000000000000000000000000B2
:10FE500000000000000000000000000000000000A2
:10FE60000000000000000024000028000000000046
:10FE700060080000000000000024000000000000F6
:10FE800028A08080000000000000000000A844803E
:10FE9000C0A0888400808080808080804084FCECCA
:10FEA0001800444480801090A4A0C004DC806C3C06
:10FEB00000446000004400800080C004C4002400AE
:10FEC00000000000000000000000C004808000006E
:10FED000A4B08080844008A0C8A480808C800000EA
:10FEE000444000808000D4F84084C00400002828EA
:10FEF000280028280000280028282824482CE8006A
:10FF00000000000090909090101010108080808071
:10FF10007C2880281450109080EC28000000C0003D
:10FF200000000000000000000000000000000000D1
:10FF300000000000000000000000000000000000C1
:10FF400000000000000000000000000000000000B1
:10FF500000000000000000000000000000000000A1
:10FF60000000000000000000000000000000000091
:10FF70000000000000000000000000000000000081
:10FF800028C0808000000000000000000000008009
:10FF9000C0A08884808080808080808020887C5879
:10FFA00000004480808008A004C0C0048CFCA858D5
:10FFB00000006000004400280080C004C40000006D
:10FFC00000000000000000000000C004000000006D
:10FFD0008080000084400000C8A400004824000085
:10FFE00000000000000080800000C004800028287D
:10FFF000280028280000280028282828282CE80085
:00000001FF
